:020000040800F2
:10000000002000103970000821270008491200085C
:100010001D27000819270008152700080000000008
:100020000000000000000000000000001127000890
:100030000D27000800000000092700081D1800080F
:10004000A1700008A1700008A1700008A17000084C
:10005000A1700008A1700008914D0008BD4E000875
:10006000814E0008454E0008094E00085D6D0008ED
:100070004D6D00083D6D00082D6D00081D6D0008D8
:10008000096D0008F56C0008A1700008A170000857
:10009000E5270008A1700008A1700008CD4D0008F8
:1000A0003D15000889150008A1700008B115000869
:1000B0007D1500086D150008A1700008A1700008EA
:1000C000A1700008A1700008A1700008A1700008CC
:1000D000A1700008CD180008A17000085118000890
:1000E000554D0008A1700008CD680008A1700008F7
:1000F0004D150008A17000085D150008A1700008EA
:10010000000000000000000000000000A1700008D6
:10011000A1700008A1700008A1700008A17000087B
:10012000E16C0008CD6C0008B96C0008A56C0008F3
:10013000916C0008A17000080000000000000000A1
:10014000A1700008A1700008A17000080000000064
:10015000000000000000000000000000000000009F
:100160000000000000000000A1700008A17000085D
:10017000A170000800000000000000000000000066
:0801800000000000A17000085E
:100188002DE9F04FB54E9DB006F1010906F1020BBD
:10019800741E002554F80B0C88B3B14BCC2707FB11
:1001A800053708E0242838D0AE4B9B7E834200F008
:1001B800D28054F80B0C03685B689847F8B154F880
:1001C8000B0C0368DB68984714F8033C002BE9D054
:1001D800012B26D0022B2AD0032B3BD0042B00F076
:1001E800A980052B43D0062BE3D114F8027C002FFD
:1001F8004ED0012F00F0EC80002304F8033C0135B9
:10020800032D06F1CC0609F1CC090BF1CC0B04F156
:10021800CC04BFD11DB0BDE8F08F012304F8033C26
:10022800C7E74D2812D0002304F8033CC1E7002398
:100238003C2804F8033C00F088803E28B9D101220C
:10024800032304F8022C04F8033CB2E7022304F861
:10025800033CAEE7C028E6D80022042304F8060CC5
:1002680004F8050C04F8072C04F8033CA1E714F87B
:10027800073C14F8062C9A4274D814F8053C8342BB
:10028800D1D114F8027C062304F8033C002FB0D126
:10029800754B14F804AC14F806ECADF82A700FCBC3
:1002A8000DF1100888E80F00631E03EB0E010FFA2A
:1002B8008AF20893BAF1380F4FF001030991ADF8AB
:1002C8002820ADF818208DF82C3000F0DD8354D9A3
:1002D800BAF1800F00F0F88300F2A280BAF1520F51
:1002E80000F04A8440F2DB81BAF1540F00F0BC847C
:1002F800BAF16E0F40F074825C4ADFF898A1128858
:10030800DAF808100093FF2A594B5A480490A8BFFE
:10031800FF2281F3100189B240461A7006F032F8C4
:100328003946404606F02EF8DAF8001001F30F01BE
:1003380089B245E014F8053C04F8040C584005233C
:1003480004F8050C04F8033C33E7032204F8023CE4
:1003580004F8032C2DE7484A484B49491160494A9B
:10036800DA6026E714F8052CF9184240013304F83E
:10037800052C04F8073C88721BE7BAF1040F00F05B
:10038800608440F28B80BAF1200F00F0AD8340F218
:100398006D81BAF1240F00F09E84BAF1280F40F065
:1003A8001F820093DFF8F0A0314B3748374ABAF87C
:1003B800001004901A60404605F0E4FFBAF80210F5
:1003C800404605F0DFFF0DF13008009B049A79E004
:1003D80014F8042C14F8063C611E0B4408916E2A8C
:1003E8004FF000010A9109930B91ADF8282000F015
:1003F8003D83B62A7FF400AF14F8012C0894042A30
:100408003FF6FAAE01A151F822F000BF9D0700089F
:10041800010200087B07000821070008950700086B
:10042800BAF1820F00F02B84C0F04D81BAF1A00F11
:1004380000F05E84BAF1FE0F40F0D281144F07F14C
:10044800080A37F8021B404605F09CFF5745F8D1CB
:10045800049A012300270DF1300833E0800B0020B7
:10046800740B0020FC15002098930008DC1C002069
:10047800181E0020191E0020FC9F002000ED00E03F
:10048800EFBEADDE0400FA051C1E002001060A01BD
:10049800E41C0020641C00209C1C0020BAF1020F00
:1004A80000F0068100F207839A4540F09981BF4B1E
:1004B800BE491F70242283F801A08A705346CA1CC3
:1004C8000DF1300854F80B0CADF81A30016805929C
:1004D800D1F820C0B5490491BCF1000F00F08F821B
:1004E800E047BDF91A30059A049954F80B0CA2EBB1
:1004F800010A0022C8F80020C8F804205246FF2A42
:100508004FF0240E4FF04D01A8BFFF2201338DF8A4
:1005180030E08DF8311000F0A7829DF81C30002BD8
:1005280014BF3C213E21BDF818308DF83210BAF1C5
:10053800FE0F8DF833208DF8343040F362824FEA95
:100548002A238DF8363003238DF835A0009307222F
:10055800414603F051FF009A9DF834309DF833105E
:100568000132022A83EA01030AD0042A9DF83510D1
:1005780008BF9DF8362083EA010304BF5340DBB26D
:10058800BAF1000F8DF80F3055DD5246049954F832
:100598000B0C03F031FFAAF1040189080AF1FF32BC
:1005A800013104989DF80F300090062A4FEA81081F
:1005B80040F368824FF0000E8446019470465CF860
:1005C800044B0EF1010E714580EA0400F7D8C0F320
:1005D800072141404B40C0F307414B400099019C23
:1005E80083EA1063C2454144A2EB0802DBB220D083
:1005F8000878002A83EA00031BDD4878012A83EA89
:100608000003DBB215DD8878022A83EA000310DDD7
:10061800C878032A83EA00030BDD0879042A83EAF1
:10062800000306DD4879052A83EA000301DD8A799B
:1006380053408DF80F3054F80B0C01220DF10F01C7
:1006480003F0DAFE54F80B0C03685B6A03B19847B1
:10065800002304F8033C002F3FF4D1AD54F80B0CF1
:1006680005F0D4FB54F80B0CB847C8E5BAF1050FF0
:1006780040F0B68040460B224D49009305F061FEDC
:10068800404608224B4905F05CFE404607224A498D
:1006980005F057FE0DF13008009B049A12E7BAF1F5
:1006A800440F40F09D80049A444F0DF1300809E74B
:1006B80040460422424900930DF1300805F041FEFE
:1006C800009B049AFEE63F4A01931168374B3E4867
:1006D800926804904FF6FF7A5145A8BF51464FF0F3
:1006E8000A0E21EAE171404683F800E089B20092DF
:1006F80005F048FE009A02EB820149005145A8BF67
:10070800514621EAE171404689B205F03BFE0DF100
:100718003008019B049AD5E6A3EB0B071D2F23781D
:1007280001930DF13008D4BF3A461E226378009336
:1007380059464046C8BF1746CDF820B008F058FDC6
:100748001CAB3B44214A00214046D2F800A003F8E4
:10075800401C06F051FC0099DAF80070019A8AF8FA
:100768000B2008448AF80A0043467F695046B84778
:1007780042E5164B1F683B6838469B689847144A01
:100788000123FF2179733B73137035E5114B012267
:100798001A7031E500F0F2FF0F4A104B00F5742093
:1007A80000F51070106000221A7025E5181E002050
:1007B8000C9700081897000824970008AD0E000849
:1007C800FC960008A01C0020191E0020F40E002032
:1007D800FA0E0020F80E002004110020F90E002067
:1007E800BAF1650F00F01181BAF1960F00F00D8192
:1007F800AAF1210ABAF1360F23D8DFE80AF041221C
:1008080022222222222229222222222222222222B9
:100818002222222222221C222222222222222222B6
:1008280022222222222222222222222222222222A0
:100838009C228C22600014F8013C08940A2B00F0DA
:10084800D682049A4FF0FF3300270DF1300839E6BD
:1008580014F8013C08940A2BF3D108A805F066FDAA
:10086800DFF81083A8F8000008A805F05FFD00274E
:10087800A8F80200049A4FF0FF330DF1300821E682
:100888001CA8AD4F14F8011C2278637840F8509DDD
:1008980079703A70BB7005F049FD089BF8801A46DC
:1008A800591C089112F8021B397108925B787B7108
:1008B800049A4FF0FF3300270DF1300802E614F8D0
:1008C800013C009304F1370133461A46013399423B
:1008D800FBD10DF130080892C446274604F1300ACE
:1008E80038687968BA68FB68E646AEE80F001037E2
:1008F8005745F446F4D13868BB88904ACEF80000D2
:10090800AEF804301378002BFCD18D4B1F78002FE4
:1009180000F01282FEE714F8013C0894FF2B90D1F6
:10092800884B22781A700896049A4FF0FF330027F4
:100938000DF13008C6E514F8012C0894032A80D874
:10094800531E81498148DBB203EB430301EB4303A8
:1009580002705978002A3FF474AF0EF1FF33DBB20E
:100968008B427FF46EAF0022C0F80220C0F8062048
:100978008272002B35D022780896012B827030D0F5
:100988006278CDF82090022BC2702AD0A278CDF8D8
:1009980020B0032B027124D0211DE2780891042B8A
:1009A80042711ED0611D22790891052B827118D0E1
:1009B800A11D62790891062BC27112D0E11DA2799E
:1009C8000891072B02720CD0082BE279427204F1CD
:1009D80008011CBF04F10902237A08911CBF837225
:1009E80008925B4B1F78002F3FF444AF04F0B0FD32
:1009F8000027049A4FF0FF330DF1300862E555499E
:100A080075E5012300930522A2E5534B4046B3F850
:100A1800201105F0B7FC514BB3F86812404689B273
:100A280005F0B0FC0021404605F0ACFC0021404632
:100A380005F091FC049B4A4A591C002704911F7039
:100A480011886429A8BF6421404605F09BFCBAF1CF
:100A5800960F00F063814046394605F093FC0DF18E
:100A68003008049A01232DE521215CE508A80894A3
:100A780005F05CFC08A805F059FC08A805F056FC30
:100A8800FFF7BABB0146B3E5364A324992F801E0AE
:100A980090780B7011782F4A117182F805E00521C2
:100AA8004FF00A0ED7709071517082F802E00DF184
:100AB8003008073206E5274902220A704B708F700A
:100AC800CA1C0DF13008FDE42749284A0988901E00
:100AD800FF29A8BFFF214FF00A0E02F8011C80F879
:100AE80000E00DF13008EDE4214ADFF84CA0009356
:100AF800D31E9AF801009AF800109AF802E002F85A
:100B0800030C59704046BAF8061083F802E00492C4
:100B180005F038FC049A9AF80410501C04901170DF
:100B2800049A9AF80510501C04901170009B049ABE
:100B38000DF13008C6E400BF741C0020FB0E002035
:100B480008110020F0150020C09500085C1900204D
:100B58002C1D0020181E0020E4010020740B00202A
:100B6800241D00201C1D0020EC1C00201A1E002043
:100B78001B1E00209C1C0020A948AA4ADFF8F0C2CE
:100B88000178C2F800C04FF0090E4FF0030C82F84C
:100B980005C09371D17182F804E002F1080C0029B4
:100BA80000F019810139C9B2DFF8C8E201EB41014F
:100BB8000EEB41014978002900F00D8190F802E020
:100BC80082F808E001290CF1010240F20C81093A8F
:100BD800C3785372022900F01B81037993720329A9
:100BE80002F10B0300F00D81A3F10B074279FA72B1
:100BF800042903F1010200F0F48082793A7305298F
:100C080003F1020200F0ED80C2797A73062903F13C
:100C1800030200F0E680027ABA73072903F104029E
:100C280000F0DF80427AFA73082903F1050200F028
:100C3800D880827A3A740DF130089A1D0027012372
:100C480040E4524640467849009305F07AFB39461D
:100C5800404605F097FB049A009B511C04911370C1
:100C6800049A0DF130082DE4704A7149901E0978F4
:100C780002F8011C122101700DF1300822E46D49BF
:100C88006D4A0878D1886D4A009302F8010C4046F5
:100C9800049205F077FB6A4A04991288DFF8D8A114
:100CA800FF2AA8BFFF22481C04900A70DAF808201F
:100CB80082F3100291B2404605F064FBDAF80010A6
:100CC80001F30F0189B2404605F05CFB049A5D49C7
:100CD800501C097828E75C4A00934046D2F8641211
:100CE80005F039FB0DF13008009B049AFFF7EABBC9
:100CF800564A00934046116805F02DFB544A404679
:100D0800116805F028FB534A4046116805F023FB9B
:100D18000DF13008009B049AFFF7D4BB049A012315
:100D2800D11804911370049AD11804911770049A79
:100D38000DF13008FFF7C6BB474B1868474B4FF01B
:100D4800010A83F800A003F0D3FF454A384682F829
:100D580000A004F089FB384604F086FB092004F063
:100D680083FB009804F080FBC246AAEB0807FFB299
:100D78000A2004F079FB384604F076FB1AF8017B68
:100D88000B2004F071FB384604F06EFB354B1868F5
:100D980003F0A4FF0DF166035345E6D1082004F0E3
:100DA80063FBA02004F060FBA02004F05DFB0020A2
:100DB80004F05AFB10F02000F6D1274B8246186841
:100DC80003F09CFF254B049A83F800A057464FF088
:100DD800FF33FFF777BB62460F460DF13008FFF788
:100DE80071BB012300270DF13008FFF76BBB1E4BC9
:100DF80020786178A278CDF820B0187059709A7070
:100E08001FE51A46002701230DF13008FFF75ABBEA
:100E1800164A012300270DF13008FFF753BB00BF26
:100E28005C190020181E0020049700081A1E0020D4
:100E3800F0150020601C0020741C0020191E0020E2
:100E4800DC1C0020101E0020740B0020ACF7FF1FD4
:100E5800B0F7FF1FB4F7FF1FE815002008110020A6
:100E680012110020C81500201C1D0020221E002081
:100E780003010602C0950008641C002038B5084D1F
:100E880000242B59CC3418461BB11B685B68984763
:100E980020B9B4F5197FF4D1002038BD012038BD40
:100EA800740B0020014B024ADA60FEE700ED00E017
:100EB8000400FA05012312211322417042710370C4
:100EC800037170472DE9F0410B78057BDB43DFB2F6
:100ED80000F1130200F11D0302F8015F9342FBD1F8
:100EE800DFF890E000F12701002203F8012F994272
:100EF800FBD114210524002647FA04F303F001036B
:100F0800002B1E4414BF4FF019084FF00A0814F0C4
:100F1800010FF6B214BFAC464FF0000C0023CA18FC
:100F280010FA82F20133434582F814C0F7D15A1EF1
:100F380092B20132013C8B18621C9BB201D0194657
:100F4800DAE716F0010F14BF19240A2400229918B1
:100F580010FA81F10132A2420D75F8D113449BB207
:100F68005A1C0344002192B21975AEF800200261A0
:100F7800BDE8F081E40D00202DE9F04FDFF890A0E6
:100F8800BAF802300B3383B01FFA83F901F1060B6C
:100F98004FF001084FF0000C002711F801EB3E4616
:100FA8004C460122A4F10B039BB2019105E00133E9
:100FB8009BB2017B29759C4208D0C518002AF6D13E
:100FC800C51801339BB29C422A75F6D10319013624
:100FD800092F019983F814C0F6B20CD0092E15D048
:100FE80008FA07F313EA0E0F14BF012200220C348B
:100FF800A4B20137D6E709F1780959451FFA89F9EA
:10100800CAD1AAF802C003B0BDE8F08F0022EEE70B
:10101800E40D00202DE9F047DFF85C80B8F80430D3
:1010280004331FFA83FC01F109094FF0010E11F88E
:10103800017B64460026231F0EFA06F29BB23A4053
:10104800C2B1B0F80CA0C51801339BB29C4285F818
:1010580014A0F5D101360434082EA4B2EBD10CF15A
:10106800200C49451FFA8CFCE1D10023A8F8043074
:10107800BDE8F0879246E6E7E40D002010B4026868
:10108800047B11680223A340194209D0064940682D
:1010980000240C7001684FF6FE7421400160536013
:1010A8005DF8044B704700BF58190020436A8269F5
:1010B80070B4D154436A0469426B0133A34228BF18
:1010C80000234362DAB1116811F0010101D070BC4C
:1010D8007047856A86699D422E44D6600BD3641B8F
:1010E800546081621368002143F0010380F84410C2
:1010F80070BC136070475D1B55608362F2E7026D38
:10110800136843F080031360E1E700BF026B10B47B
:1011180062B1036CC2684469D11A013B615C5DF835
:10112800044B08BF13460364C8B27047016A436999
:10113800C4685B5C0131A14228BF114601625DF8B9
:10114800044BD8B2704700BF436B13B190F844000A
:101158007047836A406A181AB0FA80F040097047ED
:10116800416A836A99420AD3CB1A416B026961B119
:101178004968501E0B4483420AD2C01A704702695C
:101188001144CB1A416B0029F2D1501EC01A704786
:10119800002070472DE9F0470569C3681D4028D035
:1011A8000F4606464FF000484FF00009B5FA85F3A0
:1011B80028FA03F2D2431B3B32611540042B16D8A0
:1011C800DFE803F03129211903007B6A002B32D0B4
:1011D80003F1FF3A1FFA8AFAC7F824903C6A34B13F
:1011E80023682046514698476468002CF8D1002DA2
:1011F800DCD1BDE8F0873868716B036889B298471D
:10120800002DD3D1F5E77868B16B036889B29847A8
:10121800002DCBD1EDE7B868F16B036889B2984728
:10122800002DC3D1E5E7F868316C036889B29847A7
:10123800002DBBD1DDE7F36A1FFA83FACEE700BFC2
:10124800184C08B50121022003F068FDA37903F0CA
:101258000903092B08D00021012003F05FFD0021BC
:10126800084603F05BFDFEE70F4A104B11681A6849
:101278000B68A0684FF6FE752B400B60138823F0AF
:1012880001031B041B0C138018B12922002382714F
:10129800C37102224E2103F093F9A06803F028FDE0
:1012A800D9E700BFE40D0020381D00203C1D0020B8
:1012B8002DE9F84FF02200218F48904CDFF860921A
:1012C8008F4D904E904FDFF85C8207F0B6FF8F4845
:1012D8008F49DFF854E2DFF854C2002213598342E1
:1012E80000F0FA80B3F1804F00F0F880AB4200F0D4
:1012F800F780B34200F0F680BB4200F0F5807345FA
:1013080000F0F480634500F0F380434500F0F2807C
:10131800DFF81CA2534500F0A9800AF5806A5345FE
:1013280008BF092300F0A3801432F02AD6D1DFF8D1
:10133800CC81784F784D08F1F0064FF0030A4FF052
:10134800020998F804301C09013C052C03F00F032E
:1013580000F2858037F8140040FA03F2D2077ED5F0
:101368004FF0010B0BFA03F3013B184005F04CFE5C
:101378006A4B1B5D184415EBC00470D055F830302B
:10138800674898F8081003F1384200EB922292F867
:10139800502002F01F005209022A0BFA00FB00F04D
:1013A8009480032A00F08A80012A05D1584A5848B7
:1013B80052694BEA02024261B4F804E0BEFA8EF2C6
:1013C800C2F11F0292B2D00803EB800002F00702BC
:1013D800046A92004FF00F0C0CFA02FC24EA0C0489
:1013E8000462046A01FA02F22243002402624FF006
:1013F800010C224603E0102A04F102042FD00CFA53
:1014080002F030EA0E0102F10102F4D1D3F808B07B
:101418000AFA04F1C9430BEA010BC3F808B0D3F880
:1014280008B0C3F808B0B3F804B01FFA8BFB2BEA76
:1014380000009880988880B29880186808401860E2
:10144800D3F800B009FA04F040EA0B001860D86835
:10145800102A01EA0001D96004F10204CFD108F191
:10146800140846457FF46DAFBDE8F88F082309EBF3
:10147800C3034FF0010B93F804A00AF01F034FEACF
:101488005A1ABAF1020F0BFA03F30BD0BAF1030F91
:101498000ED0DA457FF448AFD1F814A043EA0A0326
:1014A8004B6141E7D1F818A043EA0A038B613BE797
:1014B800D1F81CA043EA0A03CB6135E7144A144863
:1014C800D2694BEA0202C26176E7114A1048926972
:1014D8004BEA020282616FE70023C8E70123C6E7EF
:1014E8000223C4E70323C2E70423C0E70523BEE7BA
:1014F8000623BCE70723BAE7F00D0020CC940008C8
:10150800000400400008004000100040002C01408A
:101518000010024098940008841600209094000857
:10152800A893000800400140001400400034014026
:1015380000440140014902482CE600BF900E0020FB
:10154800004001400149024824E600BF680E00201F
:1015580000340140014902481CE600BF680E002023
:10156800003401400149024814E600BF400E002043
:101578000004004001494FF080400BE6180E00209F
:1015880010B5064C064804F10C01FFF703FE04F100
:10159800D4010448BDE81040FCE500BFE40D00207C
:1015A800002C01400044014001490248F2E500BF17
:1015B800F00D0020002C01401F4B98422CD0B0F1B8
:1015C800804F2BD0A3F59433984229D003F580633C
:1015D800984227D003F50063984225D003F580632D
:1015E800984223D003F59033984221D003F5406305
:1015F80098421FD003F58063984207D003F58063B3
:10160800984208BF092202D00020704708220B4BDD
:1016180003EBC203187970470022F8E70122F6E7C6
:101628000222F4E70322F2E70422F0E70522EEE7BC
:101638000622ECE70722EAE7002C0140A8930008FD
:101648002DE9F04FDFF830C1474A4849484E494D27
:101658008046102718F1FF38C0F08480DCF8043089
:10166800C3F30803002B5CD1EFF31183002B58D18F
:101678000B68946800BF08688342F9D1D6F80090D7
:101688004FF47A7000FB09FEAEEB040EBEFBF9FEC8
:1016980000FB03EEDCF80430C3F308034FF47A745C
:1016A8000120FBB9EFF31183E3B90B68D2F808A066
:1016B80000BFD1F800904B45F7D1D6F800B004FB35
:1016C8000BF9A9EB0A09B9FBFBF904FB0393A3EB9C
:1016D8000E03B3F57A7FBDD2DCF80430C3F30803F8
:1016E800002BDFD0EFF3118A87F31288D2F808B005
:1016F8001368DB0344BF2860D2F808B00B68D5F83C
:1017080000905FFA8AFA8AF31188D6F800A0994403
:1017180004FB0AF3A3EB0B03B3FBFAF304FB093353
:10172800D5E7EFF3118487F31288D2F8089013688D
:10173800D80303D501232B60D2F808900B682868DA
:10174800E4B284F31188D6F800A04FF47A7400EB61
:10175800030E04FB0AF3A3EB0903B3FBFAF304FB40
:101768000E3E97E7BDE8F08F10E000E00C1900206E
:10177800101900200819002000ED00E0204B5B68DC
:10178800C3F3080330B4BBB9EFF31183A3B91D4BFE
:101798001D4C1868A16800BF1A689042F9D11B4B0C
:1017A8001C684FF47A7202FB04F3591AB1FBF4F186
:1017B80030BC02FB00107047EFF31182102383F353
:1017C800128811498C680B6813F4803F104B02D0C3
:1017D800012018608C680B49D2B20D68186882F332
:1017E80011880A4B19684FF47A72284402FB01F3F6
:1017F8001B1B30BCB3FBF1F302FB0030704700BF8A
:1018080000ED00E00C19002010E000E010190020A5
:101818000819002030B4EFF31183102282F31288E4
:101828000649074C0A680748013200250A60256006
:10183800DBB2026883F3118830BC70470C190020B2
:101848000819002010E000E01D4B70B59C68236D5E
:10185800226BDD69C2B1636B2BB12B0702D5236DF7
:1018680008221A6270BD2A06F7D5A26A616A8A42FE
:101878001FD0511CA069A162825C2069266D81423B
:101888003285EAD3A362E8E7A906E4D5E26A1AB189
:10189800988C80B29047DEE7E1699B8C6069DBB287
:1018A8004E1CE6614354E169E368994228BFE2614E
:1018B800D1E7226D136823F080031360CDE700BFE2
:1018C800141900201D4B70B51C68236D226BDD694F
:1018D800C2B1636B2BB12B0702D5236D08221A62A4
:1018E80070BD2A06F7D5A26A616A8A421FD0511CC8
:1018F800A069A162825C2069266D81423285EAD3A3
:10190800A362E8E7A906E4D5E26A1AB1988C80B226
:101918009047DEE7E1699B8C6069DBB24E1CE661AB
:101928004354E169E368994228BFE261D1E7226D37
:10193800136823F080031360CDE700BF141900205B
:1019480008B51F4B002832D01E481A6800210180B4
:10195800137813F07F0316D0012B27D0022B24D144
:10196800527902F00F039B0003F1804303F5B8435B
:1019780012061B681FD403F44053B3F5805F0ED1E1
:10198800012303700BE0527A930654BF03780223B5
:1019980051064CBF43F0010323F0010303700A4BC7
:1019A8001B681B699847074808BD084608BD1B689F
:1019B80002221A8208BD03F03003102BEFD1DFE7B3
:1019C8002C180020F00E00205018002008B538B15F
:1019D800064B1B689B689847054B18680C3008BD78
:1019E800034B1B6801221A8208BD00BF5018002053
:1019F8002C18002008B538B1064B1B681B6898479F
:101A0800054B18680A3008BD034B1B6801221A826F
:101A180008BD00BF501800202C18002010B5094C34
:101A280060680368DB69984750B9237A0BB9637A11
:101A380033B160680368DB68984700232372A37298
:101A480010BD00BFF00E00204FF0FF30704700BF00
:101A58000020704700207047014BD87A704700BFBC
:101A6800F00E002010B405481E2404FB02110144A6
:101A780000200B735DF8044B704700BFF00E002088
:101A8800F0B41C7894B11E200A4F10FB02120020FB
:101A98000D181D2D07EB000500F10106D8BFAD1884
:101AA800F0B2D8BF2C731C5C002CF1D10020F0BC24
:101AB800704700BFF00E0020014B1888704700BF28
:101AC800000000200020704738B50F4C637AA3B996
:101AD800D4F81432C01A00280FDD60680B4B056873
:101AE80016210C228172C272012161726D6908216E
:101AF800A847606803685B6A9847A07A10B9207A9B
:101B080000B9607A38BD00BFF00E00203097000899
:101B180038B50B4C94F8183205460BB904F058FF49
:101B2800084B94F81D129A7894F81C3212F0400F62
:101B380014BF10220D220A441E332A726B7238BD5C
:101B4800F00E00200000002070B51F4C94F81E32E3
:101B5800ABBB94F8213203F0F7031C4E84F8213212
:101B6800306803F0C5F894F82152042003F07CFC97
:101B7800284603F079FC306803F0C0F894F8205246
:101B880094F81F323068C5F1030545EA830503F070
:101B9800AFF8EDB21024E0B203F066FC0134284639
:101BA80003F062FC202CF6D1306803F0A7F8214638
:101BB8004FF4F072064807F040FB002070BD94F81F
:101BC800213243F00803C8E7F00E0020E815002092
:101BD800FC0E00200F4B104A1B689BB223F0070332
:101BE80003EBC00002443E294FEA42020AD94B09DE
:101BF800C80604BF03F1FF339BB29B0243F40043C2
:101C0800136070474B08C90748BF01339B02136034
:101C1800704700BF505C004006300020054B064A64
:101C28001B689BB223F0070303EBC0000244520079
:101C380011607047505C00400230002000230360B0
:101C4800436083608381036143618361C36103628D
:101C580043628362704700BFF0B48B680F6A0E69F5
:101C68004D698A69CC693B4333432B434E6A8D6A7D
:101C78008F89134302682343334322F4FF422B43E3
:101C880022F070020C6813434A680360476084605E
:101C9800C260F0BC704700BF02683B494FF6FE7354
:101CA8001A4088424FF0000302600360436083607B
:101CB800C36027D0354B98422AD0354B98422DD057
:101CC800344B984230D0344B984239D0334B9842F9
:101CD8003CD0334B98420FD0324B98423CD0324BD9
:101CE80098423FD0314B984242D0314B984245D030
:101CF800304B98421ED070472F4A536843F07063A8
:101D0800536070472C4A536843F00F035360704781
:101D1800294A536843F0F00353607047264A5368D2
:101D280043F4706353607047234A536843F4704325
:101D380053607047214A536843F470235360DAE7CD
:101D48001D4A536843F47023536070471A4A536816
:101D580043F4700353607047184A536843F00F0305
:101D680053607047154A536843F0F0035360704757
:101D7800124A536843F47063536070470F4A5368BC
:101D880043F4704353607047080002401C0002404F
:101D98003000024044000240580002406C000240FB
:101DA80080000240080402401C0402403004024043
:101DB800440402405804024000000240000402406B
:101DC8002DE9F04F764C94F818328FB013B994F887
:101DD80022521DB100200FB0BDE8F08F714F724E36
:101DE8003868DFF8E081012384F8183202F080FFB8
:101DF800802003F039FB284603F036FB0546386897
:101E080002F07CFFB378D8F80020AB423DD004F054
:101E180043FE0022B4F82C32B6F800C04FF0050A91
:101E280016464FF006094FF00708E01803F1010EB7
:101E380090F83012057BA94206F1050113D004EB96
:101E4800010BA11980F83052180A81F810A481F802
:101E5800129481F8133481F8148481F81104013242
:101E680006368BF810541FFA8EF3634502F101020F
:101E78002CD2632AD9DDA4F82C325EBB00230020C3
:101E880084F818320FB0BDE8F08F484B1D78002D4C
:101E9800BFD1D4F82432D31AB3F57A7FB9D93868C8
:101EA800019202F025FFA02003F0DEFA284603F095
:101EB800DBFA8146386802F021FF19F0040F019A15
:101EC80050D0C4F82852C4F82422A2E70023A4F86A
:101ED8002C32D2E71FFA86F9E37A03F0FF05002BCC
:101EE800FAD1DFF8E480324E4046FFF7D5FE30469F
:101EF800FFF7D2FE03A8FFF7A1FE2E4A2E4B099545
:101F080003A930460A9507950B950C9505950895F4
:101F180003920493ADF81890FFF79EFE3368274D9F
:101F280043F0010333601022802303A94046059241
:101F380008930495FFF790FED8F80030386843F00E
:101F48000103C8F80030336843F00203336002F03D
:101F5800CFFE01231A4AE37293889BB243F003032E
:101F680093808BE709F00503012B11D0002BAAD130
:101F7800B3785B06A7D5D4F82812D8F8003059B141
:101F88005B1A642B9FD9019204F086FD019A9AE7A7
:101F9800B3785906EFD596E7C4F8283293E700BF1F
:101FA800F00E0020E815002000000020EC150020AD
:101FB800440002400C3800400400002000130020B8
:101FC800003800400C19002058000240084BDA681D
:101FD800D1070BD4DA68D20601D502207047DB6836
:101FE80013F0040F14BF032004207047012070472A
:101FF80000200240B64B596801F00C0104292DE974
:10200800F04100F08D81082900F07681B14A026024
:1020180001B10021DFF8B8E2AF4CDEF80430C3F3B9
:10202800031323441E7AF6B222FA06F34360DEF85D
:102038000450C5F3022525442F7A23FA07F7876051
:10204800DEF80450C5F3C22525442D7AEDB2EB40E5
:10205800C360DEF82CC04FEA1C1C0CF00F0E04EB1A
:102068004E0E1CF0100FBEF818E01FFA8EFE03D0BB
:10207800BEF1000F40F0A8809646DFF854C2C0F8C1
:1020880010E0DCF82CE04FEA5E2E0EF00F0C04EBAB
:102098004C041EF0100F248BA4B202D0002C40F088
:1020A80090801446DFF828E24461DEF830C0894C9D
:1020B8001CF0100F0CBFA4469446C0F818C0DEF8F8
:1020C80030C01CF0200F0CBFA4469446C0F81CC0BA
:1020D800DEF830C01CF0400F18BF14460462DEF86A
:1020E8003040E40502D5914200F0CC80784C436240
:1020F800D4F830E01EF4805F57D0914200F02B8175
:102108008362246BA40540F1CF80714CC362D4F87C
:1021180030E04364246B240540F1E0806C49096B8E
:1021280083646B490C6BA50752D00B6B03F0030358
:10213800012B00F007810B6B03F00303022B00F067
:1021480036810B6B03F00303032B40D0604B196BF4
:1021580011F4403F42D147635D4B196B11F4402F96
:1021680057D187635A4B196B11F4401F6CD1C76361
:10217800574B196B11F4400F00F08180196B01F473
:102188004001B1F5800F00F0E3801A6B02F44002C1
:10219800B2F5000F00F013811B6B03F44003B3F595
:1021A800400F00F0C980BDE8F0818362246BA4056C
:1021B8007AD59142A9D1AE42A7D14FEA410C6446E3
:1021C800D5E0B1FBF4F46DE7B1FBFEFE55E7414BFA
:1021D80003633F4B196B11F4403FBCD0196B01F4FA
:1021E8004031B1F5803F00F0AF80196B01F4403108
:1021F800B1F5003F00F0DF801B6B03F44033B3F50B
:10220800403F04BF334B4363314B196B11F4402FEC
:10221800A7D0196B01F44021B1F5802F00F096800A
:10222800196B01F44021B1F5002F00F0B8801B6B49
:1022380003F44023B3F5402F04BF264B8363244B9C
:10224800196B11F4401F92D0196B01F44011B1F5CC
:10225800801F75D0196B01F44011B1F5001F00F013
:10226800A2801B6B03F44013B3F5401F04BF194B46
:10227800C363174B196B11F4400F7FF47FAF0764EA
:10228800BDE8F081AE427FF431AF4FEA410CC0F8AF
:1022980024C0DEF8308018F4805F64465FD1836222
:1022A800DEF83040A4058AD4094CC362246B640567
:1022B80001D591423CD0064C4364246B24050DD5CE
:1022C80091427FF42BAFAE427FF428AF54005EE01A
:1022D8000010024000127A00000000203A4C83648B
:1022E800246BA4047FF51CAF91427FF419AFAE4272
:1022F8007FF416AF540050E059685A68C1F383411F
:10230800D50301F102010FD5DB6A304A03F00F0350
:102318000133B2FBF3F301FB03F101600A4679E6EE
:102328002A4A0260002175E6294B03FB01F1F4E714
:10233800AE42C0D14C0022E0244B0364BDE8F081DA
:10234800C26315E7026301E7426305E7826309E7B1
:102358000264BDE8F081AE427FF4D2AE4C00DFF8F3
:1023680068E08462DEF830E01EF4007F9CD0DFF87D
:1023780058E0C462DEF830E01EF4806F9BD0DFF8CE
:1023880048E04464DEF830E01EF4006FA6D00E4941
:102398008464096B8D047FF5C3AEC464C1E64FF451
:1023A80000438363DEE64FF40043C363E0E64FF483
:1023B80000430363CAE64FF400434363CCE64FF49B
:1023C80000430364BDE8F0810010024000127A0067
:1023D80000093D00F0B504460068D1F808E04B68F4
:1023E800CF680E6920F001000D46496920606268D7
:1023F80022F4405242EA0E02626022683B4322F411
:10240800B05222F00C02334313432360A36823F431
:1024180040730B4395B0A3606846FFF7EBFD174B7D
:102428009C4224D0164B9C4223D0164B9C4222D06F
:10243800154B9C420CBF0F9A109A23682968180400
:1024480048BF5200B2FBF1F301FB1322B2EB510F6C
:10245800226828BF0133120405D54FF6F0721A40DE
:10246800C3F3420313439BB2A38115B0F0BD0C9A8A
:10247800E3E70D9AE1E70E9ADFE700BF0038014075
:102488000044004000480040004C004000222DE974
:10249800F04313460F6801264FF0030E04E00133A2
:1024A800102B02F1020224D006FA03F434EA0705DD
:1024B800F5D10D7905F1FF3CBCF1010F0EFA02FCD4
:1024C80019D96FEA0C0C046804EA0C040460046867
:1024D800954025430560C568CC790EFA02FC944006
:1024E80025EA0C0501332C43102BC46002F10202CB
:1024F800DAD1BDE8F083D0F808800EFA02FC6FEA62
:102508000C0C08EA0C08C0F8088091F80580D0F88F
:10251800089008FA02F848EA0908C0F80880B0F8F4
:1025280004801FFA88F828EA040484808C79B0F8BB
:1025380004809C4044EA0804A4B28480C3E700BF36
:102548002DE9F0430368244F9B687860044689B0FE
:1025580098474FF00108FF23637384F80C80A02488
:10256800FF2C19D05FFA88F6234600257868E9B26F
:1025780001F1040E026880F80AE0C6720331D2F84D
:10258800189001340135C9B23246C847E4B2182D53
:10259800234602D0FF2CE9D1FF2408F10108B8F145
:1025A800050FDDD168460D4A0D4901F0DFF96B468C
:1025B80006221421786802F0BDFC06220D21094B81
:1025C800786802F0B7FC786803685B6A984701236B
:1025D8003B7209B0BDE8F083F00E00204097000878
:1025E800489700084C970008704700BF2DE9F04154
:1025F800304E37683A8A2AB93D7A042D43D0BC8ACE
:10260800042504E0BC8AA2428CBF0225042594421A
:1026180028BF14461FFA84F8BB6940469847264BE2
:102628001B689BB223F0070303F1005303F54053E3
:102638005B00621C1C68A4B204F1005404F5405409
:1026480052104FEA440418BF002306D030F8021B8A
:1026580024F8231001339342F8D141460020FFF7B4
:10266800DDFA7B8A3A8A1549A2EB080298443020A1
:102678004FF440533A82A7F81280376848808B801D
:102688003D72BDE8F0810D4B1978012905D0072569
:1026980010223D725A80BDE8F08107480849006859
:1026A8001A7080B220F007000144490030200A6007
:1026B8005880E5E72C180020505C00406015002089
:1026C8000230002008B50B4B002093F82C10FFF7C0
:1026D80081FA094B1B68187A082805D1074B4FF473
:1026E8008051102299805A80A0F10900B0FA80F038
:1026F800400908BD400000202C180020601500206B
:10270800704700BF704700BF704700BFFEE700BFBB
:10271800FEE700BFFEE700BF704700BF202938B5BD
:1027280003D80D4621BB284638BD2025294610234D
:10273800114A30F8024B22F8044C013B02F1040222
:10274800F7D10120FFF76AFA0C490D4A0B682B44B0
:102758000B60136823F4E04323F040039BB283F03B
:10276800300343F4004343F080031360284638BD28
:102778004B1C5B1089B2DBE7846100407C150020AC
:10278800045C0040B2B170B4541EE4B201340023BA
:1027980064001E46020F092A02F1300586BF37324F
:1027A800CA54CD54CA1802339C424FEA00105670DE
:1027B800F0D170BC704700BF064B9B7A23B9064B1B
:1027C80001221A6004F0CEBA034B05221A6004F005
:1027D800C9BA00BF3018002078150020A1490B683D
:1027E8002DE9F043A04CA14D9BB2E380E2882B88F1
:1027F8001A40970583B006D54FF6FF520A60227A31
:102808000132D2B22272E2881A40160427D4E28832
:1028180002F48062134219D1E28802F48052134212
:1028280002D103B0BDE8F0838E4A00234EF6FF7153
:1028380011602373237B052B00F27781DFE813F007
:10284800F600E600E100D600CB00B700854A884BC9
:102858004FF6FF315B68116098472B88DCE700234F
:10286800DFF80082834E844FADF80230D8F800209C
:1028780090B213044BF6BF7E48F28001E08040F12D
:10288800DC80E38803F00F039A0002F1804202F52E
:10289800B8426372002B63D13B689BB2A380A388C4
:1028A80003F030036380A38803F44053A3803B689C
:1028B80003EA0E0383F4005383F020030B433B60C9
:1028C800E388D80640F1BB803B689BB2ADF8023084
:1028D800BDF802301A0500F1D580BDF802301904A0
:1028E800C4D53B68654E40F68F721340D6F8008019
:1028F8003B6098F80830022B0AD0042B08D0032B31
:1029080000F0F281052B00F0EF81072B00F06382C5
:10291800082388F80830FFF7D5FE574B1B68A288B4
:102928004BF6BF71D204A28803EA010348BF83F4BF
:1029380080539704628848BF83F40053D6066288A0
:1029480048BF83F01003900648BF83F0200343F488
:10295800004343F08003484A9BB213602B8856E734
:10296800116889B2ADF80210BDF80210090414D438
:10297800BDF802301A067FF579AF627A930003F149
:10298800804303F5B84306EB82021968906948F65C
:102998000F720A401A60804768E7116840F68F7026
:1029A800013B014056F8233011609847E0E7637B0C
:1029B800013BDBB26373637B03F0FF02002B7FF400
:1029C80030AF2F4908684FF6EF73034006200B60BD
:1029D8002073226125E72A4A13689BB243F010034B
:1029E80005200A211360207361731AE7637B013B9A
:1029F800DBB26373637B002B7FF413AF0423237371
:102A08000FE702220323627323730AE71C4D2A6827
:102A18004FF6FB7313402B60FFF7CEFE4FF41641C1
:102A280004220123296022732361FAE62369002B1B
:102A380000F0828005232373F3E62B88E7E63A68E3
:102A48000E4E48F60F731A4033683A601A7A022A13
:102A580000F08080042A7DD0062A00F0BD8008227C
:102A68001A7258E7445C004060150020CC1D002015
:102A78004000002000940008005C00402C18002052
:102A8800405C00403B689049904E914A40F68F70F8
:102A980003403B600968336889B221F007010A44A2
:102AA800197A52000929126842D092B2520002F1F2
:102AB800804202F5C0421178197092F8018083F8BB
:102AC80001809088C1B2090241EA10215980108919
:102AD800C1B2090241EA102199809289DA80012164
:102AE8001972002A3CD0B8F1060F00F0D680B8F170
:102AF800000F7DD1598831B95A6822F47F42B2F566
:102B0800003F00F02282734F3B6840461B6998479C
:102B1800032833687ED01A8A4FF6FF718A4279D02B
:102B280002284CD108221A72F5E60623237378E6A8
:102B3800DA8893F80180D2E7674D2A684FF6FB736D
:102B480013402B60FFF738FE4FF4164206232A6025
:102B5800237366E6FFF74AFD33681A7A1A72DAE6D3
:102B68001A7812F07F0258D1B8F1090F00F01382D9
:102B7800B8F1050F00F0A581B8F1030F00F0B3819B
:102B8800B8F1010F00F0CE81524F3B6840465B69B7
:102B98009847032800F01882336800287FF45FAF55
:102BA80049494E4A096889B221F007010A4452008E
:102BB800002010603021062261801A72ABE6002ADC
:102BC800B0D093F900100029C0F2488103214FF4D6
:102BD80040521972A2809EE65A78052A00F00381B5
:102BE8003C4B1B689B689847336808221A7292E628
:102BF800B8F1080F40F0CA801A78500683D1384AD5
:102C08009A6100205882904733681A8A4FF6FF71FC
:102C18008A42D4D109221A727DE6012A00F02D8158
:102C2800022AB1D1B8F1010F00F08881B8F1030F81
:102C3800AAD1587947B220F08000820002F1804181
:102C480001F5B841002F0968B4BF01F0300101F463
:102C58004051032898D85888002895D1002993D046
:102C68009B7A002B90D002F1804202F5B842002FE7
:102C78001368C0F2E08123F4804323F070039BB211
:102C880083F4805343F4004343F080031360154BEF
:102C98001B689B699847336882E71A7857067FF460
:102CA80032AF9A780B4F012A00F08881022A00F08F
:102CB8008881032A7FF428AF3A68526A002A9FD194
:102CC8004FF0060820E700BF505C00402C18002099
:102CD800043000204C180020405C004002300020E6
:102CE800FD19000850180020D8F81830B8F81070EE
:102CF8009BB3002F00F09580B8F81420974228BFA6
:102D080017461FFA87F948469847B14AB14B1268E7
:102D1800B8F810E0B8F8121092B222F00702134483
:102D28005B00AEEB090E1A6892B27B1C02F10052EE
:102D380002F540521FFA8EF789445B104FEA4202AF
:102D4800A8F81070A8F8129007D052F8041B20F8C1
:102D5800021B013BF9D1B8F81070002F68D0002190
:102D68004FF440530846A380FEF758FFB8F81030D8
:102D7800B8F81420D6F8008030219A42618053D9DF
:102D8800002B5BD0052388F80830C2E5B8F10A0F9C
:102D98007FF4B9AE1A7802F07F02012A7FF4B3AE4D
:102DA8009A7A002A3FF4AFAE598800297FF4ABAE77
:102DB8005A68894F22F47F42B2F5803F7FF4A4AE6F
:102DC80058793B689B6998473368002800F0408130
:102DD80093F8018098E6804B1B68DB689847D6F823
:102DE8000080082395E51A7812F07F027FF4F8AE88
:102DF80093F803C0794840F60F7E036842EA01075A
:102E080003EA0E0301323B43042A40F8043BF4D1A1
:102E18007349744A4CF080030B6013681B6A984727
:102E2800DEE6B8F814304BB9032388F8083070E5AB
:102E3800B8F81430D6F80080002BF5D0644A062381
:102E480088F808301168684A89B221F007010A44F5
:102E5800520000203021106061805AE5D988019124
:102E68000198824251D95C4A01991268198292F8F4
:102E78002C109982FFF7BAFB4DE5B8F10B0F7FF4E0
:102E880083AE554FD9783A6858799369984733682B
:102E98009A7A002A3FF479AE00287FF476AE1A7940
:102EA800002A7FF472AE9B78002B7FF46EAE4D4BF8
:102EB8001B68DB68984733685979DA78D9721A73CE
:102EC8006EE693F90320002AFFF6C9AD9A78002A26
:102ED8007FF4C5AD9A88002A7FF4C1AD9A7A002A9A
:102EE8003FF45EAEBBE5DA78012A7FF44DAE9A88EE
:102EF800002A7FF449AE5A7A3A4942F0200209681A
:102F08005A72CB69984733684AE6914240F2818009
:102F18003149096891F82C60B1B291426FD9002209
:102F28002270A6E7DA78012A7FF42EAE9A88002A62
:102F38007FF42AAE5B7A9B067FF526AE05F0EAF9A8
:102F480000287FF421AE33682AE693F8008018F051
:102F58007F084DD0B8F1010F60D0B8F1020F4BD106
:102F680093F8058008F00F018A0002F1804202F50B
:102F7800B84218F0800F126814BF02F0300202F451
:102F88004052032938D818F0700835D1002A3FF488
:102F9800BAAD164A34E6DA788A423FF6F5AD997842
:102FA80000297FF4F1AD998800297FF4EDAD0D4932
:102FB8009A720B685B6898473368F1E53A68D2699A
:102FC8007CE63A68126A79E6336809221A72A2E442
:102FD800505C0040043000204C180020005C004089
:102FE8004C5C0040501800200230002049190008AD
:102FF8009A88002ACDD086E54FF0000883E592FB39
:10300800F6F006FB1022002A7FF433AF012222706B
:103018002FE7104A126892F82C102AE70D4F5879BA
:103028003B689B699847336800287FF4D1AE9A7A49
:10303800002AAED1CCE623F4E04323F040039BB250
:1030480083F0100343F4004343F0800313601EE64B
:10305800014AD5E54C180020D5190008FF20704713
:10306800012380F845307047014B1868704700BF4E
:103078007415002001207047704700BF704700BFDB
:1030880008B103487047034B1B6808221A8270472F
:10309800380000202C1800202DE9F04190F8445009
:1030A800002280F8442015B90120BDE8F081184EAF
:1030B800736813B91846BDE8F0817368052B02D010
:1030C8001046BDE8F081134FD7F8008000F13004B6
:1030D800B3682946204683B9FFF720FB3B68A3EB7A
:1030E8000803322BA5EB000504440BD8002DDBD0D8
:1030F800B36829462046002BEED03B68A3EB0803B3
:10310800322BE5D9B5FA85F04009BDE8F08100BF5A
:10311800741500200C190020002280F84520BBE718
:1031280090F844305A1C0344D2B280F8442083F803
:10313800301090F845300BB1132A00D9ACE770472E
:103148002DE9F041DFF84C80D8F804300BB9BDE820
:10315800F081D8F80430052BF9D10D4E002A144619
:103168003768F4DD0D460AE0FFF7D8FA3368DB1B51
:10317800322BA4EB00040544E9D8002CE7DDD8F88D
:10318800083021462846002BEED00020EEE700BF8D
:103198000C190020741500202DE9F041234C244E11
:1031A80082B02368002B3AD12568EFB2002D39D0C0
:1031B8000023207B1A46E11801440DF1080E013363
:1031C8007244DBB2097C02F8041CAB421A46F2D303
:1031D80023685B1B2360D4F8008038442073B8F15F
:1031E800000F06D0002DDCD09DF8040002B0BDE829
:1031F800F08140210320FEF7EDFC336884F80C8051
:1032080023F4804323F070039BB283F4405343F4C8
:10321800004343F080033360002DC2D0E4E7012768
:103228003D46C5E7207B2F46D2E700BF7415002036
:103238000C5C00402DE9F04F87B00A23BE4DBF4F0C
:10324800BF4CC04E04900393BF4B93F85010986D39
:10325800C1F3400101F058FDBB4B93F85010586D75
:10326800C94301F0010101F04FFD05230293B64B5C
:10327800DFF8D892986D01F031FDB34B586D01F02D
:103288002DFD4FF0320A4FF0100C4FF47A70D9F838
:103298000430C3F30803002B40F0CB81EFF3118314
:1032A800002B40F0C6812968A26800BF2B689942AC
:1032B800F9D1D7F800E000FB0EF39B1AB3FBFEF33D
:1032C80000FB01314FF0010E0191D9F80430C3F32E
:1032D8000803002B40F03C81EFF31183002B40F0F2
:1032E80037812B68A16800BF2A689342F9D1D7F8C3
:1032F80000B000FB0BF2521AB2FBFBF200FB0323F7
:10330800019A9B1AB3F57A7FDFD3BAF1010ABED1CD
:103318008D4BDFF83892986D01F0E0FC8A4B586DC0
:1033280001F0DCFC4FF0320A4FF0100C4FF47A70C9
:10333800D9F80430C3F30803002B40F05D81EFF3A4
:103348001183002B40F058812A68A16800BF2B68C0
:103358009A42F9D1D7F800E000FB0EF35B1AB3FBF1
:10336800FEF300FB02324FF0010E0192D9F804304F
:10337800C3F30803002B40F0C380EFF31183002B45
:1033880040F0BE802B68A16800BF2A689342F9D13B
:103398008846396800FB01FBABEB0808B8FBF1F87D
:1033A80000FB0383019A9B1AB3F57A7FDED3BAF147
:1033B800010ABDD1029B013B13F0FF0302937FF486
:1033C80056AFDFF888A14FF4FA784FF0100C4FF49D
:1033D8007A70DAF80430C3F30803002B40F0468112
:1033E800EFF31183002B40F041818E462A68A168D3
:1033F80000BF2B689A42F9D10B4671469E4600FBE6
:1034080001F3A3EB0E0EBEFBF1F100FB02124FF02D
:10341800010E0192DAF80430C3F30803002B40F0E0
:10342800CF80EFF31183002B40F0CA802B68A1688E
:1034380000BF2A689342F9D18946396800FB01FB2D
:10344800ABEB0909B9FBF1F900FB0393019A9B1A4D
:10345800B3F57A7FDED3B8F10108BAD1049BFF2B0C
:1034680040F03E814FF47A7ADFF8E09050464FF012
:10347800100CD9F80430C3F30803002B40F0138173
:10348800EFF31183002B40F00E812968A26800BF7A
:103498002B689942F9D1D7F800E000FB0EF39B1A8C
:1034A800B3FBFEF300FB01314FF0010E0191D9F897
:1034B8000430C3F30803002B66D1EFF31183002B0C
:1034C80062D12B68A16800BF2A689342F9D1D7F866
:1034D80000B000FB0BF2521AB2FBFBF200FB032315
:1034E800019A9B1AB3F57A7FE1D3BAF1010AC0D1E8
:1034F800039B013B03937FF4A7AE07B0BDE8F08FB1
:10350800EFF311818CF31288A2682368DB0344BFB0
:10351800C6F800E0A2682B68D6F80080C9B281F32B
:1035280011883968434400FB01F8A8EB0208B8FB8E
:10353800F1F800FB038335E70C190020101900206F
:1035480010E000E0081900207415002000ED00E0EC
:10355800EFF311888CF31288A1682368DB0344BF5A
:10356800C6F800E0A1682B6832685FFA88F888F32B
:103578001188D7F800801A4400FB08F35B1AB3FBE4
:10358800F8F300FB0233BBE6EFF311888CF31288E3
:10359800A1682368DB0344BFC6F800E0A1682B6874
:1035A80032685FFA88F888F31188D7F800801A44DF
:1035B80000FB08F35B1AB3FBF8F300FB02338FE759
:1035C800EFF311818CF31288A2682368DB0344BFF0
:1035D800C6F800E0A2682B68D6F80090C9B281F35B
:1035E800118839684B4400FB01F9A9EB0209B9FBC2
:1035F800F1F900FB039329E7EFF311818CF31288AB
:10360800D4F808E02368DA0303D501233360D4F83B
:1036180008E02B683268C9B281F3118839681A4406
:1036280000FB01F3A3EB0E03B3FBF1F300FB023243
:1036380099E6EFF311828CF31288D4F808E0236836
:10364800D90303D501233360D4F808E02B68316827
:10365800D2B282F311883A68194400FB02F3A3EB53
:103668000E03B3FBF2F300FB01312BE6EFF31181FC
:103678008CF31288D4F808E02368DA0303D5012311
:103688003360D4F808E02B683268C9B281F3118836
:1036980039681A4400FB01F3A3EB0E03B3FBF1F303
:1036A80000FB0232B3E6EFF311828CF31288D4F8F0
:1036B80008E02368D90303D501233360D4F808E070
:1036C8002B683168D2B282F311883A68194400FB3A
:1036D80002F3A3EB0E03B3FBF2F300FB0131E3E6C5
:1036E800954B93F85010986DC1F3400101F00CFB15
:1036F800914B93F85010586DC94301F0010101F046
:1037080003FB049BCDF80880013305938A4BDFF84F
:103718002C92986D01F0E2FA874B586D01F0DEFAB1
:103728004FF0FA0A4FF0100C4FF47A70D9F80430C1
:10373800C3F30803002B40F0E280EFF31183002B62
:1037480040F0DD802968A26800BF2B689942F9D152
:10375800D7F800E000FB0EF39B1AB3FBFEF300FB67
:1037680001314FF0010E0191D9F80430C3F3080379
:10377800002B40F08B80EFF31183002B40F0868004
:103788002B68A16800BF2A689342F9D1D7F800B026
:1037980000FB0BF2521AB2FBFBF200FB0323019A67
:1037A8009B1AB3F57A7FDFD3BAF1010ABED1624B17
:1037B800DFF88891986D01F091FA5F4B586D01F030
:1037C8008DFA4FF0FA0A4FF0100C4FF47A70D9F8CE
:1037D8000430C3F30803002B74D1EFF31183002BDB
:1037E80070D12968A26800BF2B689942F9D1D7F82F
:1037F80000E000FB0EF39B1AB3FBFEF300FB013164
:103808004FF0010E0191D9F80430C3F308030BBB44
:10381800EFF31183F3B92B68A16800BF2A689342BC
:10382800F9D1D7F800B000FB0BF2521AB2FBFBF249
:1038380000FB0323019A9B1AB3F57A7FE3D3BAF10D
:10384800010AC4D1029B059A01339A4202937FF47C
:103858005DAF07E6EFF311888CF31288A16823683F
:10386800DB0344BFC6F800E0A1682B6832685FFA42
:1038780088F888F31188D7F800801A4400FB08F309
:103888005B1AB3FBF8F300FB0233D3E7EFF31188BD
:103898008CF31288A1682368DB0344BFC6F800E0F4
:1038A800A1682B6832685FFA88F888F31188D7F81E
:1038B80000801A4400FB08F35B1AB3FBF8F300FB23
:1038C80002336CE7EFF311828CF31288D4F808E026
:1038D8002368D90303D501233360D4F808E02B68A3
:1038E8003168D2B282F311883A68194400FB02F3B6
:1038F800A3EB0E03B3FBF2F300FB013180E7EFF318
:1039080011828CF31288D4F808E02368D90303D510
:1039180001233360D4F808E02B683168D2B282F30F
:1039280011883A68194400FB02F3A3EB0E03B3FBBA
:10393800F2F300FB013114E77415002000ED00E0FC
:1039480010B5FEF743FB01280CD14FF4302400E0FA
:103958004CB1FEF73BFB012804F1FF34F8D0002CF2
:1039680008BF052010BD052010BD00BF0EB42DE90D
:10397800F04189B010AD684B019000240295039383
:1039880026465622019B591C019101341A70039B4B
:103998005A1C03921A78002A3ED0252AF2D19A1C82
:1039A800049603925878302858D00027A0F13003A5
:1039B800DBB2092B39D96C283DD0642800F09680F9
:1039C8000FD8252847D06CD9582878D06328DED15D
:1039D800019B2A78591C01911A7001340435039B04
:1039E800D6E7732853D05FD9752865D10DF114082F
:1039F8002868434600220A21043502F05FFC43464A
:103A08003A46049901A801F0DDFD039B5A1C039274
:103A18001A780444002AC0D1019B002220461A705B
:103A280009B0BDE8F04103B0704704AA03A901F04A
:103A380005FE6C28C1D1039B1A4601330393127803
:103A4800642A5BD00FD8252A05D05FD9582A11D00F
:103A5800632ABDD09CE7019B252294E7DA1C0392D8
:103A680098780127A2E7732A11D052D9752A33D042
:103A7800782A8DD1A2F158014A420DF114084A4121
:103A8800286843461021043502F018FCB7E72B6874
:103A98000499002201A801F095FD04350444039B14
:103AA80076E70028B8D072E76E287FF470AF039BE2
:103AB8002A68043514606BE778287FF468AFA0F1B2
:103AC80058035A420DF114085A41286843461021F8
:103AD80002F0F4FB043592E70DF114082868434618
:103AE80000220A21043502F0E9FB88E70DF11408E9
:103AF80028684146043502F0B3FB80E70DF114084D
:103B080028684146043502F0ABFB78E7002A83D0E9
:103B18003EE76E2ACCD03BE74997000870B5324C97
:103B2800324B23602046FEF70FF800250122FF23C1
:103B3800222022736373A57300F07EFC206110B10C
:103B48002523C5718371492100F00CFF206901F01C
:103B5800CFF86420FDF774FD206901F0CFF82C2020
:103B680000F06AFC606118B11D2200238271C371E4
:103B78000D2100F0F7FE606901F0C0F81C4A606989
:103B8800138823F040031B041B0C138013889BB27B
:103B980023F0380343F00803138013889BB243F0E3
:103BA8004003138001F0A4F8002001F05DFC02201E
:103BB80001F05AFC606901F0A1F8667FA57F237FB8
:103BC8000C492376C0220023C6F12006C5F1100552
:103BD8000320E67784F8205003F032F80248FDF716
:103BE80097FF014870BD00BFD41500203894000825
:103BF80000380040396900081C4A92F82430022B2A
:103C080030D802EBC3011846098D0133C907DBB26E
:103C180022D4032B26D002EBC30110B40C8D023042
:103C2800E407C1B218460BD4022902D1138FDB076F
:103C38000FD4032382F8243000205DF8044B70472A
:103C48000B460B4982F8243001EBC0005DF8044BA9
:103C5800704708460323F4E7054982F8243001EB4E
:103C6800C000704782F8243000207047D415002027
:103C7800FC1500202DE9F047764D95F98C308342EC
:103C88008CB00DD095F99830834200F0C18195F938
:103C9800A430834200F0D58100200CB0BDE8F08745
:103CA80000277E00F31905EB8303B3F89440002C3A
:103CB800F2D102288A4607D0142800F0CD8018B126
:103CC80020460CB0BDE8F0875FFA80F948465146B7
:103CD80001F014FB04460028F2D0006D00230322F3
:103CE800A37162710268236222F0010201210DF1C1
:103CF8000408E361A3626362E36284F84410C4F8D1
:103D080008A0414602600C22029303930493069391
:103D18000592CDF804A0FEF75DFB6079236DA179CB
:103D280000F00202002A15BF4FF440324FF48032EF
:103D38004FF4003E4FF0000E10F0010F586808BF16
:103D4800724611F0010F14BF024320EA02025A60C2
:103D58009A6809074CBF42F0080222F008029A60EC
:103D68001A68216B42F001021A60002900F0708184
:103D78004046FDF763FFE26CE3686169206B0192DE
:103D88004FF480520A92002202910B9280210592F0
:103D98000792089203922022ADF8103009920691FA
:103DA800FDF77AFF4146206BFDF756FF226B236D26
:103DB800116841F001011160996841F04001996072
:103DC800526892B22264626B002A00F03C8140463D
:103DD800FDF734FFA26C236901924FF480524FF033
:103DE800000A606B0A92ADF8103080221023069208
:103DF8000393CDF82CA0CDF814A0CDF81CA0CDF8D5
:103E080020A0CDF824A0FDF747FF4146606BFDF7E1
:103E180023FF626B236D116841F002011160C2F843
:103E280004A0C2F804A09A6842F080029A601A6856
:103E380042F0010220461A603E4405EB8605012344
:103E480080F80490C5F89000A5F894300CB0BDE84F
:103E5800F08700BFD4150020DFF818928048D9F801
:103E6800183043F00103C9F81830112100F07AFD29
:103E78007B4800F03DFF01F07FF9794800F03EFFF4
:103E8800D9F814300DF1040843F40033C9F814309C
:103E98004FF4C05E0322022341464FF090408DF854
:103EA8000A408DF80B40CDF804E08DF809208DF814
:103EB8000830FEF7EBFA4FF0904395F85422586A11
:103EC800DFF8D0C1DFF8D0E1664C674920F47040D4
:103ED8005862586A40F460405862586A20F470206A
:103EE8005862586A40F4602058624FF48023CCF836
:103EF8000030DEF800305D4823F48023CEF800302F
:103F0800236802F1804223F48023236002F5823281
:103F180001244FF0080E4FF0120CC5F850C285F876
:103F280055E285F85642136843F480231360D5F8A8
:103F3800503223F01F0E03F01F035EF8012004FA2D
:103F480003F322EA03034EF80130D5F8503223F088
:103F58001F0E03F01F035EF8002004FA03F322EAA1
:103F680003034EF8003095F85522D5F85032102A40
:103F780050D002F1804223F01F0102F5823203F093
:103F88001F03885804FA03F303438B50384A39490E
:103F9800394BC5F8783200241460CA693748C5F827
:103FA800580242F40002CA614FF0020A03F13002DB
:103FB800C5F87C221B6885F864A29847304B314AC3
:103FC800DA604FF00109142340468DF804308DF86B
:103FD80005A08DF806408DF8079001F071F99DF85D
:103FE80007308DF805902A228DF806408DF80420B8
:103FF80053B9254B4FF48062C3F88420234B6B647C
:104008004FF01409224817E7404601F059F9F5E73F
:10401800012746E623F01F0203F01F0352F801E0D0
:1040280004FA03F343EA0E035350D5F8503223F051
:104038001F0203F01F03115804FA03F30B43135034
:10404800A4E702272DE61A6842F080021A60EEE61D
:1040580020221A621A6842F020021A60B3E600BFF2
:10406800E416002004040140080401400C04014047
:10407800D8004242001002404000002030180020C2
:1040880000ED00E00005FA0500E100E06494000896
:104098001816002014040140000401400F4B1A8D2B
:1040A800D1074FF000000AD41A8ED2070FD4188F08
:1040B80010F001000ED1032283F824207047024635
:1040C8000121074883F8241000EBC2007047022141
:1040D8000122F6E703210222F3E700BFD4150020EE
:1040E800FC15002010B50A4C2422002104F18C0094
:1040F80005F0A3F8142000210222032384F88C0081
:1041080084F8981084F8A42084F8803210BD00BF89
:10411800D41500204348444A018D4B0830B403F0BD
:1041280077338D08CB1A05F03335CC0804F01134F9
:104138005B1B1B1B03EB231303F00F3382FB0342B0
:104148001A44D211C2EB02229A1A012A01F0010480
:1041580005DD022A63D101F0810181295FD1058E35
:104168006908EA0701F077314FEA9502A5EB0101EA
:1041780002F033324FEAD503A1EB020203F0113308
:10418800A2EB030303EB2313274A03F00F3382FB4D
:1041980003121A444FEAE212C2EB022248BF01346A
:1041A800A3EB020248BFE4B2012A05DD022A36D198
:1041B80005F08105812D32D1058F690801F077312D
:1041C800AA08EB07A5EB010102F033324FEAD50349
:1041D800A1EB020203F01133A2EB030303EB231359
:1041E800114A03F00F3382FB03121A444FEAE2121A
:1041F800C2EB022248BF0134A3EB020248BFE4B27B
:10420800012A05DD022A0AD105F08105812D06D192
:10421800601E02288CBF0020012030BC704700209F
:10422800FBE700BFD415002081808080036B43B179
:10423800026C5B6893422FBF981AC0689B1AC0181B
:104248007047C269036A9A422FBFD01AC0688018A3
:10425800C01A70471A232B22837219230370027322
:1042680000232A22037582708375704700231F225A
:10427800027043708370C370704700BF30B5044646
:10428800006D61710368A26823F00103036087B0C1
:10429800A379009213F004023DD04FF4805213F03A
:1042A8000203019244D102934FF4806300220393E6
:1042B80011F00103059237D1049308238D0769464D
:1042C80048BF0493FEF786F86079236DA17900F062
:1042D8000202002A15BF4FF440324FF480324FF4E7
:1042E8000034002410F0010F586808BF2246CC079C
:1042F8004CBF024320EA02025A609A6809074CBF81
:1043080042F0080222F008029A601A6842F001029C
:104318001A6007B030BD13F0020301920BD04FF4BE
:10432800005513460295C1E7042304930C23C5E7FF
:104338004FF40053B7E70293B8E700BF10B504463F
:10434800006DA160036823F001030360A37986B0C0
:1043580013F00402009141D04FF4805213F002038D
:10436800019244D102934FF4806362790393D10799
:104378004FF000030493059345BF042304930823D7
:104388000C236946920748BF0493FEF723F8607927
:10439800236DA17900F00202002A15BF4FF44032C4
:1043A8004FF480324FF40034002410F0010F5868A5
:1043B80008BF2246CC074CBF024320EA02025A60DB
:1043C8009A6809074CBF42F0080222F008029A6076
:1043D8001A6842F001021A6006B010BD13F0020319
:1043E800019207D04FF4005113460291BDE74FF4F4
:1043F8000053B7E70293B8E703682DE9F041DF6996
:104408001FB13B46BDE8F0411847002A164611DDAA
:1044180004460D460E4400E023689B6820469847F2
:104428000028F9D0236815F8011B1B682046984717
:10443800AE42F1D1BDE8F08110B50409013C052C6C
:1044480017D80D4B33F8142000F00F0042FA00F390
:1044580013F001030DD0012303FA00F001381040D6
:1044680002F0D2FD054A064B125D104403EBC00072
:1044780010BD002010BD00BF98940008909400085B
:10448800841600202DE9F04F4A484B4B4B4C4FF017
:1044980090414FF0010A4FF002094FF004084FF025
:1044A800080C4FF0100E20274026802530F8022BEC
:1044B80012F0010F03D01960A3F804A0083312F01A
:1044C800020F03D01960A3F80490083312F0040F08
:1044D80003D01960A3F80480083312F0080F03D042
:1044E8001960A3F804C0083312F0100F03D0196044
:1044F800A3F804E0083312F0200F02D019609F805F
:10450800083312F0400F02D019609E80083312F071
:10451800800F02D019609D80083312F4807F05D087
:104528004FF4807B1960A3F804B0083312F4007FBD
:1045380005D04FF4007B1960A3F804B0083312F4D7
:10454800806F05D04FF4806B1960A3F804B008336E
:1045580012F4006F05D04FF4006B1960A3F804B093
:10456800083312F4805F05D04FF4805B1960A3F81C
:1045780004B0083312F4005F05D04FF4005B1960F3
:10458800A3F804B0083312F4804F05D04FF4804BE1
:104598001960A3F804B00833D20B04D04FF40042DA
:1045A80019609A80083301F58061A1427FF47EAFDB
:1045B800BDE8F08F98940008841600200018004881
:1045C800002867D003682DE9F04F03F138445C4EAA
:1045D800A40A0125345D04F01F066409022C05FABB
:1045E80006F558D0032C00F0A580012C58D08088FF
:1045F800B0FA80F4C4F11F04A4B2E50803EB850502
:1046080004F007042E6AA4000F27A74026EA07062D
:104618002E622E6A01F00307A2407C1E3243012C51
:10462800C1F3810CC1F300182A62C1F341113CD9CE
:10463800C60700F18980850700F19580440700F1DD
:10464800A380020700F1B180C60600F1BF8085068D
:1046580000F1CD80440600F1DB80020600F1E9801C
:10466800C60500F1F780850500F10581440500F1D4
:104678001381020500F12181C60400F12F81850410
:1046880000F13D81440400F14B81020400F159819D
:10469800BDE8F08F70472B4CA6693543A561A6E7A6
:1046A800284C666935436561A1E7002422464FF02E
:1046B800010E4FF0030904E00132102A04F102044C
:1046C800E6D00EFA02F636EA0005F5D1D3F808A0CE
:1046D80009FA04F5ED430AEA050AC3F808A0D3F875
:1046E80008B00CFA04FA4AEA0B0AC3F808A0B3F8AF
:1046F80004A01FFA8AFA2AEA06069E80B3F804A0E4
:1047080008FA02F646EA0A06B6B29E801E682E40ED
:104718001E60D3F800A007FA04F646EA0A061E60EF
:10472800D3F80CA001FA04F605EA0A0A46EA0A05D3
:10473800DD60C1E7034CE6693543E56157E700BF33
:10474800F8930008001002401A6822F003021A6069
:104758001A683A431A60DA6822F003020A438507A6
:10476800DA607FF56BAF1A6822F00C021A601A68DB
:1047780042EA87021A60DA6822F00C0242EA8102F1
:104788004407DA607FF55DAF1A6822F030021A60DC
:104798001A6842EA07121A60DA6822F0300242EA1E
:1047A8000112DA6002077FF54FAF1A6822F0C002E3
:1047B8001A601A6842EA87121A60DA6822F0C002A0
:1047C80042EA8112C606DA607FF541AF1A6822F420
:1047D80040721A601A6842EA07221A60DA6822F4FC
:1047E800407242EA01228506DA607FF533AF1A6823
:1047F80022F440621A601A6842EA87221A60DA686C
:1048080022F4406242EA81224406DA607FF525AF4D
:104818001A6822F440521A601A6842EA07321A608B
:10482800DA6822F4405242EA0132DA6002067FF581
:1048380017AF1A6822F440421A601A6842EA8732AF
:104848001A60DA6822F4404242EA8132C605DA6028
:104858007FF509AF1A6822F440321A601A6842EAF2
:1048680007421A60DA6822F4403242EA01428505BA
:10487800DA607FF5FBAE1A6822F440221A601A68E3
:1048880042EA87421A60DA6822F4402242EA814208
:104898004405DA607FF5EDAE1A6822F440121A601A
:1048A8001A6842EA07521A60DA6822F4401242EAA9
:1048B8000152DA6002057FF5DFAE1A6822F4400281
:1048C8001A601A6842EA87521A60DA6822F44002CB
:1048D80042EA8152C604DA607FF5D1AE1A6822F046
:1048E80040721A601A6842EA07621A60DA6822F0AF
:1048F800407242EA01628504DA607FF5C3AE1A6845
:1049080022F040621A601A6842EA87621A60DA681E
:1049180022F0406242EA81624404DA607FF5B5AE73
:104928001A6822F040521A601A6842EA07721A603E
:10493800DA6822F0405242EA0172DA6002047FF536
:10494800A7AE1A6822F040421A601A6842EA8777CE
:104958001F60DA6822F0404242EA8171D960BDE8FE
:10496800F08F00BF002852D0036803F138422DE9C8
:10497800F04F920A504DAA5C02F01F05520901241B
:10498800022A04FA05F443D0032A00F09080012A91
:1049980043D001F003077A1E012AC1F3810CC1F349
:1049A80000188088C1F341113CD9C60700F18880FE
:1049B800850700F19480440700F1A280020700F106
:1049C800B080C60600F1BE80850600F1CC804406A2
:1049D80000F1DA80020600F1E880C60500F1F680F1
:1049E800850500F10481440500F11281020500F1FA
:1049F8002081C60400F12E81850400F13C81440425
:104A080000F14A81020400F15881BDE8F08F704737
:104A18002A4A95692C439461BBE7284A55692C4377
:104A28005461B6E7002422464FF0010E4FF0030907
:104A380004E00132102A04F10204E6D00EFA02F66C
:104A480036EA0005F5D1D3F808A009FA04F5ED43D4
:104A58000AEA050AC3F808A0D3F808B00CFA04FA61
:104A68004AEA0B0AC3F808A0B3F804A01FFA8AFAA6
:104A78002AEA06069E80B3F804A008FA02F646EA77
:104A88000A06B6B29E801E682E401E60D3F800A0AB
:104A980007FA04F646EA0A061E60D3F80CA001FAE3
:104AA80004F605EA0A0A46EA0A05DD60C1E7034A90
:104AB800D5692C43D4616CE7F893000800100240D4
:104AC8001A6822F003021A601A683A431A60DA6810
:104AD80022F003020A438507DA607FF56CAF1A6893
:104AE80022F00C021A601A6842EA87021A60DA6831
:104AF80022F00C0242EA81024407DA607FF55EAFD9
:104B08001A6822F030021A601A6842EA07121A601C
:104B1800DA6822F0300242EA0112DA6002077FF511
:104B280050AF1A6822F0C0021A601A6842EA871267
:104B38001A60DA6822F0C00242EA8112C606DA6018
:104B48007FF542AF1A6822F440721A601A6842EA86
:104B580007221A60DA6822F4407242EA01228506C6
:104B6800DA607FF534AF1A6822F440621A601A6876
:104B780042EA87221A60DA6822F4406242EA812215
:104B88004406DA607FF526AF1A6822F440521A60AC
:104B98001A6842EA07321A60DA6822F4405242EA96
:104BA8000132DA6002067FF518AF1A6822F4404233
:104BB8001A601A6842EA87321A60DA6822F44042B8
:104BC80042EA8132C605DA607FF50AAF1A6822F434
:104BD80040321A601A6842EA07421A60DA6822F418
:104BE800403242EA01428505DA607FF5FCAE1A6878
:104BF80022F440221A601A6842EA87421A60DA6888
:104C080022F4402242EA81424405DA607FF5EEAEA2
:104C18001A6822F440121A601A6842EA07521A60A7
:104C2800DA6822F4401242EA0152DA6002057FF59E
:104C3800E0AE1A6822F440021A601A6842EA875203
:104C48001A60DA6822F4400242EA8152C604DA6045
:104C58007FF5D2AE1A6822F040721A601A6842EAEA
:104C680007621A60DA6822F0407242EA016285043B
:104C7800DA607FF5C4AE1A6822F040621A601A68DA
:104C880042EA87621A60DA6822F0406242EA816288
:104C98004404DA607FF5B6AE1A6822F040521A6012
:104CA8001A6842EA07721A60DA6822F0405242EA49
:104CB8000172DA6002047FF5A8AE1A6822F0404259
:104CC8001A601A6842EA87771F60DA6822F0404261
:104CD80042EA8171D960BDE8F08F00BF30B1026847
:104CE8008388918A0B4218BF1B049361704700BFE9
:104CF80010B1036882881A85704700BF10B1036835
:104D080082889A61704700BF38B100298388026899
:104D180014BF002110218B409361704710B4094BD8
:104D2800094A1C7801238340234052F8200029B9FE
:104D3800B3FA83F149095DF8044BE5E7191C18BF7C
:104D48000121F8E7C4150020C81500202DE9F0411D
:104D58000B4E346873691C400FD0DFF82880012798
:104D6800B4FA84F3C3F11F0307FA03F558F82300D4
:104D780003689847AC437561F2D1BDE8F08100BF84
:104D880000040140781800202DE9F0410B4E3468EA
:104D980073691C400FD0DFF828800127B4FA84F328
:104DA800C3F11F0307FA03F558F82300036898476F
:104DB800AC437561F2D1BDE8F08100BF0004014049
:104DC800781800202DE9F0410B4E346873691C40B7
:104DD8000FD0DFF828800127B4FA84F3C3F11F034A
:104DE80007FA03F558F8230003689847AC43756140
:104DF800F2D1BDE8F08100BF00040140781800201E
:104E08002DE9F0410B4E346873691C400FD0DFF870
:104E180028800127B4FA84F3C3F11F0307FA03F5C6
:104E280058F8230003689847AC437561F2D1BDE890
:104E3800F08100BF00040140781800202DE9F041FE
:104E48000B4E346873691C400FD0DFF828800127A7
:104E5800B4FA84F3C3F11F0307FA03F558F82300E3
:104E680003689847AC437561F2D1BDE8F08100BF93
:104E780000040140781800202DE9F0410B4E3468F9
:104E880073691C400FD0DFF828800127B4FA84F337
:104E9800C3F11F0307FA03F558F82300036898477E
:104EA800AC437561F2D1BDE8F08100BF0004014058
:104EB800781800202DE9F0410B4E346873691C40C6
:104EC8000FD0DFF828800127B4FA84F3C3F11F0359
:104ED80007FA03F558F8230003689847AC4375614F
:104EE800F2D1BDE8F08100BF00040140781800202D
:104EF8000D490E4B8A6942F0010210B58A611A68A1
:104F08000B4C42F400621A601A6842F480521A602C
:104F180020464022002104F090F94FF0FF3323642B
:104F2800C4F8433010BD00BF00100240000001402B
:104F3800781800202DE9F041044618460D4616461B
:104F4800984602F059F82768E6722844A072294664
:104F58007D69434632462046AC46BDE8F04160478D
:104F68002DE9F0473E4ADFF800E13E484FF00A0CD1
:104F780010254FF47A740127DEF80430C3F30803D0
:104F8800002B50D1EFF31183002B4CD15668816868
:104F980000BF53689E42F9D1D2F8088004FB08F399
:104FA8005B1AB3FBF8F304FB063ADEF80430C3F3EC
:104FB8000803EBB9EFF31183D3B95368D0F808802D
:104FC80000BF51688B42F8D1D2F8089004FB09F170
:104FD800A1EB0808B8FBF9F804FB0383A3EB0A0369
:104FE800B3F57A7FE1D3BCF1010CC5D1BDE8F087F8
:104FF800EFF3118885F3128886680368DB0344BFE2
:1050080017608668516813685FFA88F888F3118812
:10501800D2F808800B4404FB08F1891BB1FBF8F1B6
:1050280004FB0313DAE7EFF3118185F31288D0F854
:1050380008800368DE0344BF1760D0F8088053680F
:105048001668C9B281F3118891681E4404FB01F304
:10505800A3EB0803B3FBF1F304FB063AA5E700BF93
:105068000819002010E000E000ED00E02DE9F0470D
:105078003E4ADFF800E13E484FF0190C10254FF486
:105088007A740127DEF80430C3F30803002B50D1EB
:10509800EFF31183002B4CD15668816800BF536829
:1050A8009E42F9D1D2F8088004FB08F35B1AB3FBDF
:1050B800F8F304FB063ADEF80430C3F30803EBB94F
:1050C800EFF31183D3B95368D0F8088000BF516853
:1050D8008B42F8D1D2F8089004FB09F1A1EB08083B
:1050E800B8FBF9F804FB0383A3EB0A03B3F57A7F53
:1050F800E1D3BCF1010CC5D1BDE8F087EFF311880D
:1051080085F3128886680368DB0344BF17608668E6
:10511800516813685FFA88F888F31188D2F8088014
:105128000B4404FB08F1891BB1FBF8F104FB0313E2
:10513800DAE7EFF3118185F31288D0F80880036865
:10514800DE0344BF1760D0F8088053681668C9B2F8
:1051580081F3118891681E4404FB01F3A3EB080353
:10516800B3FBF1F304FB063AA5E700BF08190020DA
:1051780010E000E000ED00E02DE9F0473E4ADFF8DE
:1051880000E13E484FF0C80C10254FF47A7401270F
:10519800DEF80430C3F30803002B50D1EFF311837A
:1051A800002B4CD15668816800BF53689E42F9D1E4
:1051B800D2F8088004FB08F35B1AB3FBF8F304FB8E
:1051C800063ADEF80430C3F30803EBB9EFF31183B2
:1051D800D3B95368D0F8088000BF51688B42F8D122
:1051E800D2F8089004FB09F1A1EB0808B8FBF9F81C
:1051F80004FB0383A3EB0A03B3F57A7FE1D3BCF185
:10520800010CC5D1BDE8F087EFF3118885F312884A
:1052180086680368DB0344BF1760866851681368B3
:105228005FFA88F888F31188D2F808800B4404FBE9
:1052380008F1891BB1FBF8F104FB0313DAE7EFF37C
:10524800118185F31288D0F808800368DE0344BF13
:105258001760D0F8088053681668C9B281F31188BE
:1052680091681E4404FB01F3A3EB0803B3FBF1F3BD
:1052780004FB063AA5E700BF0819002010E000E08B
:1052880000ED00E000F01F0240090123022803FAA4
:1052980002F30ED0032807D0012800D07047074A30
:1052A80051690B4353617047044AD1690B43D36179
:1052B8007047024A91690B4393617047001002409E
:1052C80030B40C4B0178DA6843780B4CD243C2F304
:1052D8000222C2F10402934060181B0101F01F056D
:1052E80001224909DBB2AA4080F8003344F82120A2
:1052F80030BC704700ED00E000E100E0554B2DE9BF
:10530800F04303EB800383B0DC68002C00F0888056
:10531800656D514F4FF4807304F5AD7206466868A9
:10532800A16004F15A01276020656161A261E36010
:105338002361287EFFF7A6FFEF68FFB1DFF824E1BD
:10534800002371464868874201F11C0103D00133EC
:105358000C2BF7D10023C3EBC3030EEB83033F48A9
:105368001A6941694FF00C0E1143721C416183F8B0
:1053780018E05A76236D27632433E364AF683FB39C
:10538800DFF8E0E0002271464868874201F11C011D
:105398005ED001320C2AF7D100221046C2EBC202BD
:1053A8000EEB8202DFF8B4E01769DEF814302C49FE
:1053B8003B43CEF814300B27731C53761776EA7EDE
:1053C800234601F03DFC236DAA6862632833A36479
:1053D80094F85900FFF730F8074694F85800FFF79B
:1053E8002BF895F81990804647B10B22731CBA71B7
:1053F800FB7138464A462E21FFF7E2F8B8F1000F54
:105408000AD001360C2388F807604A4688F8063027
:1054180040462E21FFF7D4F8236B2BB1636B1BB1E9
:10542800204603B0BDE8F0832B7FAA7E8DF80420C8
:105438009B090021012201A88DF805308DF806107E
:105448008DF80720FFF73CFF204603B0BDE8F08346
:10545800D0B2A3E708190020A49400080010024065
:10546800DD6800089400002040F2E933104900E0AC
:10547800B3B10A89013B12F0020F9BB2F8D00D4B71
:105488000B49187040F2E93300E04BB10A89013B3F
:1054980012F0010F9BB2F8D0064B1878C0B27047D3
:1054A800054A538F01339BB25387508FC0B2704760
:1054B800003800400C3800400819002010B52DEDC8
:1054C800028B9FED218A20EE088A0446B0EE480A36
:1054D80003F026F8F0EE408AB0EE480A02F0D8FF52
:1054E800F7EE007A9FED197AF0EE675AE8EE875AE0
:1054F8000023A361B0EE676AC7EEA56A6361236201
:10550800E361A3626362A8EEC76ABDEC028B77EE23
:10551800C07AB6EE007AF8EE005A27EE877A20EEC7
:10552800250A27EE267A26EE266A66EEA77A20EE68
:10553800260A84ED046AC4ED017A84ED007A84EDCC
:10554800027A84ED030A10BD7CD9A03EF304353FEE
:105558000B4890F850305BB1D0F84833013300E085
:105568000B4690F85020591C002AF9D1C0F848334E
:10557800D0F8443303491B6801F10A00184700BFFB
:10558800081900205E19002050B1202809D02128D0
:105598000ED024280ED025280ED018280ED0002092
:1055A80070470023064803EB830300EB8300704732
:1055B8000123F7E70223F5E70323F3E70423F1E7E1
:1055C800CC940008F0B51C78002A0CBF4FF0200ED0
:1055D8004FF0300E5D1C4CB300292BDD2E4601E048
:1055E8001146AAB116F8017B4A1E002FF8D18E1E6B
:1055F80072B13146046801394A1C671C002A0760E9
:1056080084F800E0F6DC1C7826EAE6714A1C5CB1F6
:10561800D21A0368591C01601C70AB1815F8014BAD
:10562800002CF6D11846F0BD1346FBE7002903DC31
:105638002346F7E70022EBE74E1EDAE7F0B40D68E1
:1056480000240BE0052B18D8A0F137030A2B14DC33
:1056580004EB840415F8010B03EB4404A0F13003B8
:10566800DEB2092EA0F16107F2D9052FA0F141039E
:10567800E8D8A0F157030A2BEADD0D601460F0BCEE
:10568800704700BF002302220271037043708370C9
:10569800C3707047024B1A889B78028083707047EA
:1056A800BC9500083A4B1A784AB15A7E19691861B4
:1056B800012A08D002D3042A00D8704700225A6071
:1056C8009A60DA60704770B493F82720B3F93E40C7
:1056D80093ED1D6AD3ED157AD3ED1E6A93ED143A56
:1056E800B3F93C50D3ED115A93ED187ADFED293A0E
:1056F80093ED174AD3ED164A03EB420240F6E4460F
:10570800928E92B205EE102A06FB02F2B8EE455AC6
:10571800401AC4EB12324FF47A7101FB02F292FB89
:10572800F5F202FB00F0A5EE036A83B0DA64E5EE59
:10573800276A9A6007EE900AF8EEE77A27EE467A2B
:10574800E7EEA35AFCEEC67AE6EE446ACDED017A9E
:10575800F0EE477ABDF80420C3ED1D6AE5EE247A21
:1057680006FB02F2C4EB1232BDEEE57A01FB02F24F
:10577800C3ED1E7A92FBF5F2C3ED115A9A645A6092
:1057880083ED107A83ED037A03B070BC704700BFD5
:10579800601C00202FE33E3170B4344B1A7E012A7E
:1057A80083B013D00022A3F87C20A3F87E2093F8BE
:1057B8008020022A07D1B3F87E10B3F87C20A3F822
:1057C8008410A3F8862003B070BC704793F8222099
:1057D800D3ED2D6A93ED244AD3ED254A93ED2E7A25
:1057E800D3ED287A93ED275AD3ED265A93F8BC10B7
:1057F80093F8BD0093F8BE5003EB420201EB41144D
:10580800928E92B206EE102AB8EE466A44F6FB76FD
:10581800E6EE046AC0EB003004FB0262A6EE247ACE
:10582800B2FBF0F2B2FBF5F267EEE67AFCEEE64A7E
:10583800A6EEC57A92B2A3F88E20CDED014AE6EE27
:10584800257ABDF80410A3F87E2004FB0161B1FBA2
:10585800F0F1B1FBF5F189B283ED2D7AC3ED2E7A23
:10586800A3F88C10A3F87C10A1E700BF601C0020EF
:105878000A4BD3F8C01081B110B4D3F8C8406422E1
:10588800002002FB04F25DF8044BB2FBF1F2C3F80E
:10589800C000C3F8C800A3F8C4207047601C0020EB
:1058A8002D4B93F8CC2012B193F8CD2002B9704754
:1058B8002DE9F043294C227802F0FF0E002A48D146
:1058C800D3F8D020821A002A43DB254A25491578C7
:1058D800D3F8D460DFF89880013D6F0007EB050C22
:1058E80001EB4C0C3D4401EB0609BCF8082099F883
:1058F80018C001EB4501A8FB0282C9882578D208A7
:10590800013602FB0CF208440E2E0244C3F8D460A0
:10591800C3F8D02088BFC3F8D4E035B11248026874
:10592800217801320029FBD102601048D3F8D82031
:10593800D3F8DC10008A01250023257050604B62E3
:105948000B889BB22B430B8013682B431360BDE875
:10595800F083BDE8F08300BF601C002058190020C8
:105968005C190020BC950008501C00206819002014
:10597800CDCCCCCC70B40F4C0F4E054607CC0023D1
:10598800AA60344628606960042200E0A27912F017
:10599800200F04F1140404D101330C2BF6D170BC90
:1059A800704703EB830306EB83031B79EB7270BC30
:1059B800704700BFE4950008CC940008F0B40023B9
:1059C8000C4A0361142702260125522464218360AE
:1059D800836187704360C360436186740580847601
:1059E80083720183C0F80320C0F80B20C0F813208D
:1059F800F0BC7047050405002DE9F04F7A4D81B0E1
:105A0800FBF7BCFED5F8E4400022C5F8E020002CE6
:105A180000F0AA80237D052B074617D9216A236940
:105A28000B44C31A9342B8BF05F1E4010ADBD8E07E
:105A3800137D052B0AD9136A12691344FB1A002B2C
:105A480080F2CF8051F8042F002AF1D14FF0010BDA
:105A580000231E46C5F8E03098469A4625E0636A5A
:105A68002169227DFB1AB3FBF1F301331FFA83F995
:105A780012FB09F20132013692B2B6B2A4F81890BC
:105A8800E282904507D2BBF1000F02D1B9F1010FB4
:105A980064D99046A246D5F8E030013305EB83027D
:105AA800C5F8E030D2F8E4406CB3A268CAB1B4F8E3
:105AB8001690B9F1000FD2D1216A3846791A904769
:105AC800E8B195F81831002B58D1227D676201366C
:105AD80001324FF00103B6B22383E2824FF001098D
:105AE800CFE7236A2269FB1AB3FBF2F31FFA83F9A3
:105AF800A4F81890B9F1000F27D1E28AC1E7A4F8F9
:105B08001890E28ABDE7D5F8C020D5F8C830C5F8A6
:105B180028A101321E44C5F8C020C5F8C860BAF1F2
:105B2800000F28D0DAF8203095F81821AAF8164086
:105B3800FB1ACAF81C30CAF820709ABBDAF80C3085
:105B4800384601B0BDE8F04F1847227D12FB09F234
:105B58000132013692B2B6B2E28292E7237D062B79
:105B680004BF9046A24696E7D5F8C030C5F828414C
:105B78000133C5F8C03001B0BDE8F08FFBF7FEFD7A
:105B880005F58E710EC9C01BA1EB5111834201446A
:105B9800024438BF0346C5F81C11C5F82021C5F8D2
:105BA800243192E7FBF7EAFDDAF80C30044698470F
:105BB800FBF7E4FDDAF82C20DAF82830DAF83010B0
:105BC800001B9042A3EB53130344014438BF104613
:105BD800CAF82830CAF83010CAF82C0001B0BDE85D
:105BE800F08F4FF0000B33E7601C00202DE9F041E7
:105BF8003B4ED6F82C510B2D55DC002D6EDDD6F81A
:105C0800E43098424FD0012D39D0D6F8E830984288
:105C180049D0022D33D0D6F8EC30984243D0032D2A
:105C28002DD0D6F8F03098423DD0042D27D0D6F8A4
:105C3800F430984237D0052D21D0D6F8F830984264
:105C480031D0062D1BD0D6F8FC3098422BD0072D2A
:105C580015D0D6F80031984225D0082D0FD0D6F8A7
:105C6800043198421FD0092D09D0D6F8083198423E
:105C780019D00B2D03D1D6F80C31984213D0D6F891
:105C8800E4404CB3237D017D8B420FD3154F002494
:105C98003A4605E052F8043F53B11B7D8B4207D3C7
:105CA8000134A542F6DA0020BDE8F0810D4F00244A
:105CB800631C9B00191F2A1B06EB84048046394489
:105CC800F8189200013503F09EFAC4F8E480C6F88B
:105CD8002C510120BDE8F081024FE9E7CFD0E2E77F
:105CE800601C0020441D00200D2838B55DD00B280D
:105CF8005AD8434B342202FB003021B1C36813B198
:105D0800BDE8384072E73F4DD5F82C41002C4BDDFB
:105D1800D5F8E43098425AD0012C45D0D5F8E8306F
:105D2800984256D0022C3FD0D5F8EC30984252D049
:105D3800032C39D0D5F8F03098424ED0042C33D00B
:105D4800D5F8F43098424AD0052C2DD0D5F8F83043
:105D5800984246D0062C27D0D5F8FC30984242D03D
:105D6800072C21D0D5F8003198423ED0082C1BD002
:105D7800D5F8043198423AD0092C15D0D5F8083115
:105D8800984236D00A2C0FD0D5F80C31984232D030
:105D98000B2C09D0D5F8103198422ED00C2C03D0FA
:105DA800D5F81431984204D038BD164BD3F82801E1
:105DB800A3E70C2293001448A21A191D014492006B
:105DC8001844013C03F01FFAC5F82C4138BD0022E5
:105DD800F0E70122EEE70222ECE70322EAE70422D9
:105DE800E8E70522E6E70622E4E70722E2E70822D9
:105DF800E0E70922DEE70A22DCE70B22DAE700BF48
:105E0800E4010020601C0020441D00202DE9F04F13
:105E180083B0484C484F0190019803685B699847E4
:105E2800002840F08380DFF818914448D9F80430FE
:105E3800DFF810E1C3F308034FF00A0A4FF0100C23
:105E48004FF47A75002B3BD1EFF31183002B37D138
:105E58000168A26800BF03689942F9D1DEF80060C2
:105E680005FB06F39B1AB3FBF6F305FB013101268C
:105E78000091D9F80430C3F30803002B3BD1EFF3AA
:105E88001183002B37D10368A16800BF02689342D1
:105E9800F9D1DEF800B005FB0BF2521AB2FBFBF2A7
:105EA80005FB0323009A9B1AB3F57A7FE1D3BAF175
:105EB800010AB1D0D9F80430C3F30803002BC3D0CA
:105EC800EFF311828CF31288A6682368D90302D5F0
:105ED80001233B60A66803683968D2B282F311884F
:105EE800DEF80020194405FB02F39B1BB3FBF2F319
:105EF80005FB0131BBE7EFF311888CF31288A16829
:105F08002368DB0344BF3E60A16803683A685FFA10
:105F180088F888F31188DEF800801A4405FB08F336
:105F28005B1AB3FBF8F305FB0233BBE703B0BDE82C
:105F3800F08F00BF10E000E0081900200C190020C5
:105F480000ED00E010190020152303701623C3701C
:105F5800172383712D2343702E2303712F23C371BD
:105F6800704700231B68FFDE03685A1C0260197023
:105F780070470023262203600270272282700122C4
:105F88004360027183717047F8B5574C0601A71931
:105F98000546387AFFF776F93B7A03F01F015B096B
:105FA8000122022B02FA01F278D0032B71D0012BC7
:105FB80067D0A31901351879FEF73EFAEDB2074606
:105FC80010B11223C5718371A3195879FEF734FAF9
:105FD80010B11323C5718371A3199879FEF72CFAB0
:105FE80010B11423C5718371A5190E21EA793846B9
:105FF800FEF7E6FA6879FEF71FFAEA790E21FEF74E
:10600800DFFAA879FEF718FAEA790E21FEF7D8FA2E
:10601800A359364A934251D0354A934259D0354A0A
:10602800934240D03444227B002A2FD101200224FD
:106038009A8822F480521204120C9A80998889B2A4
:1060480041F4805199801A8802F4415242F4457211
:10605800024322431A809A8822F470621204120CB6
:1060680042F4E0629A809A8B22F400621204120CC5
:1060780007219A8319821A8892B242F040021A8044
:10608800F8BD1D4B996A0A439A6292E700200446BC
:10609800CEE7194B19690A431A618AE7164BD96882
:1060A8000A43DA6085E702F5EA32116941F40041F2
:1060B8001161116921F400411161B3E702F56042F1
:1060C800D16841F48051D160D16821F48051D16008
:1060D800A8E702F5EC32116941F4804111611169B8
:1060E80021F4804111619DE728190020003001400A
:1060F80000380040003C00400010024010B40B493A
:10610800002301E0272B0CD011F8132082424FEA1C
:10611800430403F10103F5D121445DF8044B4878A9
:10612800704700205DF8044B704700BFF0950008E9
:106138002DE9F341056906460F467DBBD0F800807E
:10614800C8F30A0323B30023D6F800800193FDF7B0
:10615800F7FB042819D1224C236943F0010323617A
:10616800BBB2A8F80030FDF7EBFB04282ED108F1EC
:1061780002030193019B3F0C1F80FDF7E1FB23699C
:10618800042823F00103236125D06FF0010505E001
:10619800FDF7D6FB042805D04FF0FF35284602B09E
:1061A800BDE8F0810E4C236943F002032361C4F873
:1061B8001480236943F040032361FDF7C1FB236981
:1061C800042823F002032361BDD0E5E7236923F007
:1061D80001032361D9E7336804333360DEE700BF86
:1061E80000200240F8B504460D468E180027B54237
:1061F80001D12069F8BDE368591CE160234415F812
:10620800012B1A720429F2D1A1682046FFF790FFEA
:10621800E7602061EBE770B5448806460D46C4F395
:106228000B0422460021284603F007F833690A4A7E
:10623800934209D3094A934206D222462846194670
:10624800BDE8704002F0D4BF23B121462846BDE81E
:106258007040184770BD00BFB49D0008D29D00086B
:10626800002870B51EDB0928044620DD012303EB56
:1062780083035B00B0FBF3F2092AF8D87BB10E4E1A
:10628800B4FBF3F00928CCBF57223022A6FB03E564
:10629800024403FB1044EB0801F8012BF0D1002362
:1062A8000B7070BD2D230B7040420131DBE730309D
:1062B80001F8010BF3E700BFCDCCCCCC884230B459
:1062C8004FF001042ED301FB04F4B0FBF4F58D422A
:1062D800F9D284B1AAB901E0B0FBF4F5092DCCBF1D
:1062E800572230222A4404FB150003F8012BB4FB83
:1062F800F1F4002CF0D100221A7030BC7047B0FBCA
:10630800F4F5092DCCBF372230222A4404FB1500AE
:1063180003F8012BB4FBF1F4002CF0D100221A7021
:1063280030BC70470546002AEBD1D7E70368591CF3
:106338001A46016012F8021B0260587841EA0020F0
:10634800704738B504460068154602F051FF2268C8
:106358002A44226038BD03685A1C026010B41970C0
:1063680003680A0A5C1C04601A7003680A0C5C1C47
:1063780004601A700368090E5A1C026019705DF8EF
:10638800044B704703685A1C026019700368090AB5
:106398005A1C0260197070470A44914251D030B4B7
:1063A80041F2210411F8013B80EA0320430010F474
:1063B800004F84EA03059BB2ADB208BF1D466B00CF
:1063C80015F4004F84EA03009BB280B208BF184658
:1063D800430010F4004F84EA03059BB2ADB208BF36
:1063E8001D466B0015F4004F84EA03009BB280B28F
:1063F80008BF1846430010F4004F84EA03059BB217
:10640800ADB208BF1D466B0015F4004F84EA0300C7
:106418009BB280B208BF1846430010F4004F84EACC
:1064280003059BB2ADB208BF1D466B0084EA0300AA
:1064380015F4004F85B298B218BF28468A42B1D1E8
:1064480030BC704770B5184C23789F2B2AD16378DD
:10645800BE2B27D105221549A01C02F0F6FE08BB69
:10646800214607224FF6FF70FFF796FF104E0734BC
:1064780022884AB1A518B54214D2052A12D9214654
:10648800FFF78AFF2C46F3E721460222FFF784FF35
:106498000222A118FFF780FF41F60F53C31A584292
:1064A800584170BD002070BD00F00308A89700088F
:1064B8000000040809B10220704701288CBF02209F
:1064C800002070470B4B1B68DA78042A06D8598AD3
:1064D80030B1094B53F83200084470470020704728
:1064E80010B4054C04EBC2025DF8044B9288511AB3
:1064F800198270472C18002054040020064B1B6892
:106508005A8A18B1054B186A104470470349898C98
:106518008A1A1A82704700BF2C18002054040020E1
:10652800064B1B685A8A18B1054B986A1044704785
:106538000349898D8A1A1A82704700BF2C180020D7
:1065480054040020074B1B681B7803F07F03212BA2
:1065580001D00220704700F0DF00022814BF02209B
:10656800002070472C180020212804D0202803463A
:1065780011D0022070470F4B1A68137803F07F037D
:10658800212BF6D10C4910B5002491615482204684
:106598008847204610BD074A1268117801F07F012C
:1065A800212903D0054A0220137070470348044983
:1065B8000370E8E72C180020CD650008CA1D0020EC
:1065C80089300008FCF75CBD704700BF034B1A78A0
:1065D800202A04BF00221A70704700BFCA1D00207D
:1065E800014B04221A60704778150020034B9B7AF0
:1065F80013B1034B05221A60704700BF3018002002
:10660800781500200D4A0E4B12680E4992B222F0FE
:10661800070213445B001B68C3F309030B600B6894
:106628009BB201335B1007D00749084A52F8040BA4
:1066380021F8020B013BF9D1704700BF505C0040C4
:106648001E300020741500208415002020620040B0
:10665800014B00221A6070477C1500202DE9F04F8D
:106668006A4BDFF8D0811A68694DDFF8CCB1DFF8E2
:10667800CC9168496848DFF8C8A1684F83B0002406
:10668800C02353729472D4720193C8F800402A68E8
:1066980002EA0B0242F4007292B22A602A6802EA05
:1066A800090292B248F2800682F0100232432A6050
:1066B800D8F8002092B222F0070211444900402283
:1066C8000A60D8F80010009289B221F0070101F1A0
:1066D800005101F5405149004FF0800EC1F800E02B
:1066E800D5F800E090F82C1040F60F6000EA0E0094
:1066F800304328602046FBF76DFA29684848DFF8E0
:1067080044E1019B009A01EA0A0189B281F44051EF
:1067180031432960016801EA0B0189B20160D8F8A8
:10672800001089B221F007018E444FEA4E0E11463F
:10673800CEF8003003683B4ADFF80CE103EA0903AE
:106748009BB283F0200333430360036803EA0A0320
:1067580033439BB203601368334803EA0B0343F4E3
:10676800C0639BB21360D8F800309BB223F00703D4
:106778009E444FEA4E0E4FF48073CEF800301368F3
:1067880003EA0A0333439BB21360136803EA09035D
:106798009BB283F02003334313603B6803EA0B0B7F
:1067A8001FFA8BF33B60D8F800309BB223F0070345
:1067B800184440004FF4887303600320FBF70AFA7B
:1067C8003B6803EA0A039BB283F4405333433B60BC
:1067D8003B6803EA090333439BB22A4620463B60E1
:1067E800314640F60F75136840EA01042B4001302A
:1067F8002343042842F8043BF5D10C490C4B802074
:10680800012208601A6003B0BDE8F08F2C18002040
:10681800005C004004300020400000200C5C004078
:10682800045C0040085C00401C3000204C5C0040C8
:1068380078150020505C00408F89FFFFBF8FFFFF55
:106848008FBFFFFF0830002010300020F8B5134A32
:10685800134B10681B68C0180AD0124B12491C68E9
:106868000822FBF78FFF204604221049FBF78AFF16
:106878000F4B104A19681048104D114C00238B72A9
:1068880001274FF416414FF4E05617601360036078
:1068980016600360698011602360F8BDACF7FF1FC4
:1068A800B4F7FF1FB0F7FF1F8604002096040020EE
:1068B8002C180020405C0040445C0040CA1D0020A9
:1068C80078150020024B4FF480221A60704700BFF1
:1068D8001404014030B490E81200057B4369022299
:1068E800AA404A602268586A996A4FF6FE752A409B
:1068F8008842226004D1012283F8442030BC7047CA
:106908009C695A6B0C44D4600DD818690024411A4C
:1069180051609C621168002041F0010183F8440035
:1069280030BC11607047411A51609862F2E700BFAD
:10693800F8B50568037B2A6802269E4032420DD1CD
:10694800296804229A40114218BF6A6029680822FF
:1069580002FA03F3194218BF6B60F8BD1749184AC9
:106968000B684FF6FE7423400B6013899F07FCD514
:10697800134B1A891406FCD41B89D90718D411495A
:106988000F4A0B684FF6FE773B400B606E609388AA
:1069980023F0030304461B040B481B0C9380006878
:1069A800FEF7ACF9094A2568237B00211170C7E777
:1069B800034B9A891A89D207E1D5FAE744000240C5
:1069C8000038004058000240E8150020FB0E002067
:1069D8002DE9F84F294A137803F0FF04002BFAD168
:1069E800274FDFF8A8803868DFF8A490254D0123E9
:1069F80088F80030FEF77CF90520FEF735FD2046C3
:106A0800FEF732FD0620FEF72FFD2046FEF72CFD8F
:106A180099F80060042046F00106FEF725FD30468F
:106A2800FEF722FD2B8893B1DFF868A0164E1AF8FE
:106A380004B00720FEF718FD5846FEF715FD1AF8B2
:106A480004202B8832550134A4B2A342EFD8072082
:106A5800FEF70AFDFF20FEF707FD99F80040042025
:106A6800FEF702FD2046FEF7FFFC3868FEF746F900
:106A7800002388F80030BDE8F88F00BFFB0E002027
:106A8800E815002000000020201100200811002037
:106A980011110020FC0E00202DE9F041474E30680E
:106AA800FEF726F9464B1B78012B78D05FD3022BD3
:106AB8000AD1DFF82C81082388F800300D254FF41F
:106AC800C373404F3B8010E0DFF814813D4F98F8C6
:106AD800003003F04003002B14BF4FF4F0734FF461
:106AE800C3733B8014BF10250D25002404F110004A
:106AF800C0B2FEF7B9FC01340120FEF7B5FCA3B221
:106B0800AB42F3D398F800402F4D0020FEF7ACFCC1
:106B18002046FEF7A9FC2D4B1C780220FEF7A4FCAA
:106B28002046FEF7A1FC2A4B1C780320FEF79CFCAC
:106B38002046FEF799FC274B1C7804200443FEF7F7
:106B480093FC2046FEF790FC3068FEF7D7F83A88A9
:106B58002148002102F071FB2B7833B11F4B1B78C1
:106B680033B300232B70BDE8F081BDE8F081A0208D
:106B7800FEF77AFC0020FEF777FC00F00603022BF4
:106B8800DFF85C8007D000F00500012803D1482316
:106B980088F8003008E0082388F800308EE7DFF82E
:106BA8004080482388F8003010254FF4F07388E7B8
:106BB800FFF70EFF00232B70BDE8F081E8150020D9
:106BC800EC15002000000020A0040020F315002090
:106BD800F4150020111100202011002008110020B8
:106BE80002000020F0B5064683B00D4600240127B8
:106BF80014E003290CBF03220122C3F3011E6946D6
:106C0800C3F3810330468DF805208DF806E08DF832
:106C18000730FBF73BFC0134102C0FD02B8807FA08
:106C280004F21342F7D0AB78E9780092022903F016
:106C380003028DF80420DCD10A46DEE703B0F0BD7C
:106C480070B50F4C0F4DC0EBC00004EB80046869B1
:106C580026693043686182B09209667BA16000258D
:106C6800012101A863618DF804608DF805208DF875
:106C780006508DF80710FEF723FB02B070BD00BF69
:106C880094000020001002400348D0F83C3113B1B2
:106C980000F59A7018477047940000200348D0F810
:106CA800203113B100F58C7018477047940000200C
:106CB8000348D0F804310BB1FC301847704700BFC7
:106CC800940000200348D0F8E8300BB1E0301847B2
:106CD800704700BF940000200348D0F8CC300BB1B7
:106CE800C4301847704700BF940000200348D0F80C
:106CF800B0300BB1A8301847704700BF940000208F
:106D08000348D0F894300BB18C301847704700BF57
:106D1800940000200248836F0BB170301847704709
:106D2800940000200248C36D0BB1543018477047D7
:106D3800940000200248036C0BB1383018477047A4
:106D4800940000200248436A0BB11C301847704772
:106D5800940000200248836803B11847704700BFB9
:106D6800940000201749184B184A194810B4D1F854
:106D7800884044F47004C1F888401C6844F0010459
:106D88001C605C6822405A601A6822F0847222F4FF
:106D980080321A601A6822F480221A605A6822F433
:106DA800FE025A60DA6A22F00F02DA621A6B0024D5
:106DB80010404FF0006218639C608A605DF8044BD5
:106DC800704700BF00ED00E0001002400CC07FF8E3
:106DD800CCFC00FFF0B4594A594B5A4C1288198818
:106DE800E578511AAA4201F1020049D3217891426B
:106DF80046D39978032961D053480078022800F0D7
:106E08008F8001291A807DD075D3022904D1D888B2
:106E1800904201D201219970627A002A47D0E28813
:106E2800002A44D049480078002840D048489FEDBF
:106E3800496AD0ED026A07EE902AF8EEE66AB8EEE3
:106E4800677AF8EEE77A77EE666A66EE866A86EE25
:106E5800A77AFDEEC77A17EE902A002A66DB642A25
:106E68006ADC002A62D0D2B2A07A904234BF0022F3
:106E78000122914238BF1146DA701972F0BC70478E
:106E8800B2EB450FB5DC9978032909D00428B3D8AB
:106E98002E480021032501709980D9809D70DD70EE
:106EA80029490978022944D01A800321B4E7DA78FD
:106EB800914238BF11461972F0BC70470428EFD8C8
:106EC800214D217892FBF1F1013108291F482F78D3
:106ED800A6786578A8BF0821017089B216FB01F66B
:106EE80015FB01F5022F4FF000019E80DD8099709F
:106EF800D97016D01A809988E07A091A8A4289DDF1
:106F0800002189E7D888E57A401B824205DD988808
:106F1800904281D2002199707EE7022199707BE727
:106F28000A480D4D0078E880A9806AE70222DA70E5
:106F3800BEE706480321F4E7642295E7DC1C00203D
:106F4800081E0020741C0020E01C0020601C00208B
:106F5800641C00200000C842E41C00201F4B20488D
:106F680070B53422012500211D7002F066F91D4A12
:106F78001D491E4C1E4800230B601360FEF736FEA9
:106F880029460520FEF7B0FE2579291C4FF0070099
:106F980018BF0121FEF7A8FE6679311C4FF00800E2
:106FA80018BF0121FEF7A0FE237A0BB9617A19B147
:106FB80095B9311C18BF01210920FEF795FE0D4B2C
:106FC800D9680A20C1F34051FEF78EFE01210B203B
:106FD800BDE87040FEF788BE0121EDE7781D00206E
:106FE800441D00208C1D0020401D0020741C002022
:106FF800E4010020081E0020034613F8012B002A94
:10700800FBD1181A01387047430803F05533C01AEA
:10701800830803F0333300F03330184400EB1010CA
:1070280000F00F3000EB002000EB0040000E70472E
:1070380011481249026800608A4218D0002103E012
:107048000F4B5B58435004310E480F4B42189A427D
:10705800F6D30E4A02E0002342F8043B0C4B9A4256
:10706800F9D3FFF77FFE00F019F87047FEE70948EB
:10707800D0F800D040680047FC9F0020EFBEADDE8E
:10708800D29D000800000020880600208806002005
:10709800181F002000D8FF1FFEE700002DE98048D8
:1070A800BF4BC04AA3B01968914200AF00F0BA873D
:1070B800BD49BE4B00224FF47000C1F888003A6207
:1070C8007A621A6842F480321A6003E03A6AB2F5CA
:1070D800A04F09D01A6802F400327A623A6A013283
:1070E8003A627A6A002AF1D0B04B1B6813F4003375
:1070F80018BF01237B627B6A012B00F06887AA4DC9
:10710800AA4BAB4AEA605A6A5A6AAA4EDFF8F4A256
:1071180042F080725A625A6907F1880442F4FC020C
:1071280041F6FF715A6124F8501D032321464FF0A0
:10713800904087F83A30FFF755FD4FF6FF73214628
:107148009D483B87FFF74EFD21469C48FFF74AFDC7
:1071580021469B48FFF746FD21469A48FFF742FD26
:1071680021469948FFF73EFD2046FAF743FFBB6BDF
:107178009649974AA1FB031396499B0C0B60F02094
:1071880007234FF0000E566085F82300C2F808E088
:107198001360FDF777F9FFF755F98F4B9B460028E9
:1071A80000F0D2838D4DDA4526D2DFF85892DFF809
:1071B8005882C7F814B0A24646463488321984B1BA
:1071C800AA420ED2052C0CD9B9F800307188C3F345
:1071D8000B03994200F09A80164634883219002C25
:1071E800EED1D9F804104846FFF715F87B6909F184
:1071F80014099945E0D35446FCF78CFF002800F0A9
:107208005D84774D774B78491B7895F8B804774EAD
:10721800774A0870DFF8F491DFF8F4817148126852
:10722800F178DFF8D0B1C9F8002043F0010303700A
:1072380088F800104FF0010A16F8010B002840F0FA
:107248009E80CBF800000AF1010ABAF1040F0BF195
:10725800040BF1D198F80010664BC943186801F087
:107268000101FDF751FD98F80010624B81F0020111
:107278005868C1F34001FDF747FD98F800105D4BD1
:1072880081F004019868C1F38001FDF73DFD0121FB
:107298000220FDF743FDFDF72BFE6420FAF7D0F935
:1072A800FAF706F82320FDF7C7F8C5F8BC0418B1AB
:1072B800112200238271C3710121FDF753FBD5F818
:1072C800BC04474DDFF84CB1FDF712FD4A4B2A4686
:1072D80019201A21002603F1110E03F114080BEBF3
:1072E800060C29B19CF80AA08A4508BF82F85810F4
:1072F80028B11BF80610814208BF82F85900C6451C
:1073080029D01EF8011B9EF80300EAE77379990754
:107318007FF462AFD9F8041096F804B04846FEF737
:107328007AFFB9F80030BBEB133F0DD1B9F8023042
:10733800D9F80400A21FC3F30B039A4206F1060111
:10734800A8BF1A4601F054FF7B6909F11409994551
:10735800FFF432AF4FE7B2F8581029B12749536507
:1073680041F8262002F517722549994254D093F81E
:10737800206093F8301093F834002033ABE7FDF722
:107388005BF80121CBF800005FFA8AF328B14FF0CF
:1073980005028271C371DBF80000FDF7E3FA52E7DA
:1073A800FC9F0020EFBEADDE00ED00E000100240C3
:1073B8000005FA053F1901000004004800080048CC
:1073C800000C0048001000480014004883DE1B43EE
:1073D80010E000E010190020B49D00080000040827
:1073E80088060020EA0D0020E01C0020C4180020B8
:1073F800D80D0020C8150020A092000814190020FC
:10740800C0920008889C000807F00308141E00209A
:10741800C4150020E8180020FCF764FEDFF88CB1E2
:107428005B4BDFF88CE17C61BBF1000F30D013F9C6
:10743800082C58491144100191F8038091F806C0AE
:1074480054490EEB00068C5C1946022211F801AB78
:10745800A24591F801A008BF3471C24591F803A074
:1074680008BF86F80580E24508BF86F806C0013ADD
:10747800ECD10EEB00010E7956B14E7946B18E79FA
:1074880036B14EF800B09E79D8790A73CE71087279
:10749800414A1033934202D053F804BCC4E72C206D
:1074A8007C69FCF7C9FF30B12C2100228171C271BF
:1074B8002021FDF757FA0020FEF766FDDFF8F4B04B
:1074C800364E0120FEF760FD4FF0000A7C60002E6A
:1074D80047D01BF90B8C4FEA880303EB080EBB60FF
:1074E8002F4B03EB08042F4BA2787A612C4A12F831
:1074F80008203A614FEA8E002A4A034442F82EA037
:107508002A18FA60C3F804A0C3F808A0C3F80CA0AE
:10751800C3F810A0ABF1030414F8013B3A69934295
:107528002ED0A3787A69934223D05C45F4D1BB6806
:10753800434405EB8303D3F8C80490B1D3F8CC04D3
:1075480078B1174AC3F8C4649044ABF10B0098F8BB
:10755800044098F8062083F8D04483F8D124C3F86F
:10756800C004114B0BF1100B5B4525D05BF8076C81
:10757800ADE71046FCF760FFFB68C3F8CC04D4E71E
:107588001046FCF759FFFB68C3F8C804C9E700BFF9
:10759800E8920008C01D002018930008005400401D
:1075A800AC1D0020480B00203B9300080030014030
:1075B800281900201B930008D5F8C0347C68002BDC
:1075C80068D0987BD5F8C464D5F8C8A4D5F8CC841D
:1075D800FDF758FEB74B9E4200F0A481B64A136BE4
:1075E80023F0100313631022B3490B6B13430B638F
:1075F800BAF1000F05D0152201238AF806208AF86F
:10760800073095F8D134002B0CBF1E213E2150467F
:107618000422FCF7D5FFB8F1000F05D0162201238C
:1076280088F8062088F8073095F8D134002B0CBF6D
:107638001E213E2140460422FCF7C2FF326895F81D
:10764800D0549E4B9E489F4922F001023260326816
:10765800002D18BF034611403160336132680023A2
:1076680042F001023260B360F360B360B36843F480
:107678000043B36033683360736823F0784323F4BE
:1076880000437360336823F400333360336843F096
:10769800010333608C4B8D4A5D791E79D9F800005F
:1076A8008B4BA5F10101A6F1010EB1FA81F149094F
:1076B800BEFA8EFE4FEA5E1E012E11714FF00001D8
:1076C800196082F800E05960C0F3C03E9960D96043
:1076D800196100F4004008BF517882F802E008BF41
:1076E800197008B1D178D973917909B1D1799972A2
:1076F800012D08BF5279764E08BF5A710023B24651
:1077080098464FF0070B01259AF80000002840F032
:10771800A3800BF1010B5FFA8BFBBBF10B0F0AF196
:10772800050AF1D1002B40F0B4806A4D01210846CA
:10773800FDF7F4FA00210846FDF7F0FA00210220CF
:10774800FDF7ECFA0A26644B5868FDF7C7FA624B56
:107758001868FDF7C3FAFDF789FCFDF787FC013EC1
:10776800F1D131463046FDF7D9FA31460120FDF70F
:10777800D5FA4FF419723146584801F05EFDFCF70E
:107788008DFC4FF0CC0A18B92EE0D6B2022E2BD8B9
:107798000AFB06F8514B53F80830721C002BF4D141
:1077A800C2787B614E4B90F9020003EB8202D2F85B
:1077B8009010FCF75FFA834606EB460000EB0010DA
:1077C800BBF1000F0CD07B691946444BCC2203EB6C
:1077D800800001F032FD414B013643F808B0F6B2A3
:1077E800FCF70AFA0028D1D1FCF798F908B1FAF7A2
:1077F800A7FED9F800309B0200F17E8139493A4A48
:107808003A4D3B4C3B4803230B70002111802E4A14
:107818002B701279384B2170012A01801980598008
:1078280000F06081284B354A5979354800230129F1
:1078380003701360536093607BD0324B1B68C9F8A8
:107848000030FFF78BFB304B2F4A1B7863F07F0328
:107858001370FEF7D1F8FCE7FCF7EEFD132118B121
:10786800002380F806B0C371FDF77CF89AF8000091
:10787800FEF744FC072308F101028AF802808AF81F
:1078880004308AF801008AF803505FFA82F801236D
:107898003FE7094B0F4DDA6A22F4F872DA62DA6AC6
:1078A80042F4D872DA623C20FDF7ECFC17482A460D
:1078B800002331E000580040001002407A25E00023
:1078C800300E5000FFE0CF00741C0020E80E0020AE
:1078D800801C002094000020C8150020740B002094
:1078E800A09200080A1E00200C1E0020101E002076
:1078F800601C00200E1E0020DC1C0020641C0020E0
:107908000B1E0020D80D0020EA0D002008000240C0
:1079180001330C2B00F0A0835168814202F11C0254
:10792800F6D19AE38149824A0B6B23F020030B635B
:107938005AE6804A9FED800A80481360536093603E
:10794800D360FDF7BBFD78E79A4509D255461E4638
:10795800696828461435FEF75EFCB542F8D3B3468D
:10796800774B784DDFF804923D6101221A81764BFE
:10797800EB1ABB6003237B610026D846724BA660D6
:10798800E66026616661BB63BB68FB63D9F81030AB
:10799800180606D56D4BC9F8043003F18833C9F8C9
:1079A8000430012387F84C309F203423C9F80C3069
:1079B8005322BE234F2187F83000462087F8313004
:1079C80087F832203323072287F8331087F83400EA
:1079D80007F13001204687F8353087F83660FEF722
:1079E80001FC072207F130014FF6FF70FEF7D4FCC7
:1079F800C2450546424633D2DFF87481FA60B8F8CA
:107A080002B0B8F8003087F82D60CBF30B0BC3F346
:107A18000B000BF106011B0B06223985788507F14F
:107A28002801204687F82C30FEF7DCFB2846062282
:107A380007F12801FEF7B0FCD8F8041005465A46AD
:107A48002046FEF7CFFBD8F8041028465A46FEF722
:107A5800A3FCFB6808F1140898450546CFD398465F
:107A6800022207F11C012046BE83FEF7BBFB02225F
:107A780007F11C012846FEF78FFC43BADB430222BC
:107A880007F1280120463B85FEF7ACFB786C0028FF
:107A980040F0D382B86C97F84C30E3B998B93D6997
:107AA800C346FEF7CFFC00287FF47DAB0520FBF72B
:107AB800C1FB274B274ADA60FFF775BB2048FDF763
:107AC8007DFFFFF79EBB7B69013B7B617FF456AF6F
:107AD8003D69C346EAE7D9F8103043F08003C9F896
:107AE8001030DBE730221C4801F0A7FBB7EE000A94
:107AF8001A48FDF7E3FC95E6194B93F80BA01B78A1
:107B0800BAF1000F07D0022B00F0A683032B00F078
:107B18009A83012B2ED0134B00221A70124B124A53
:107B28001B7843F00803137068E600BF001002409A
:107B380020000010A01C0020CDCCCC3EB01C0020A2
:107B4800FC1500200000040800F003082301674525
:107B580000ED00E00400FA05EC1C0020F01C0020F9
:107B68005C1900202C1D0020EA0D00200020024096
:107B7800889C0008B94EBA48BA49337018224FF4A5
:107B88003473C6F8E4027260B16006F114001A4654
:107B98000021336101F051FB5046FDF7F5FCDFF899
:107BA800F882C36802687861C8F80020002B00F0EA
:107BB80015815046FCF740FCAB4B186018B12922E0
:107BC80000238271C3717B694E211A7AFCF7F8FC95
:107BD8007B69A64A187C5369A549C0EBC00E05EB22
:107BE8008E0EDEF810502B435361002529222B46B8
:107BF8008EF818208EF81950C022FFF721F8D8F80F
:107C08000000F9F7D9FCFDF73DFBB08899499A4A7D
:107C1800D8F8003001FB00F1914208DC02EB510575
:107C2800B5FBF1F5013DADB2691CB2FBF1F2DFF82D
:107C38006CC21988B068B2FBF0F26345C2F34E0E0D
:107C4800A6F80CE092B289B200F0BD818B4883425D
:107C580000F0B981B3F1804F00F0B581A0F59830FC
:107C6800834200F0B08100F58060834200F0AB8170
:107C78008348834200F0A38100F58060834200F0CE
:107C88009E8121F4407100F58C3089B283421980BD
:107C9800DA621D8500F09081784A934200F08C8169
:107CA80002F54062934200F0878102F580629342B8
:107CB80000F0828102F58062934200F07D8101210B
:107CC8007A695961D0797A6910F0040E527917BF30
:107CD80000254FF4807529464FF0040E00F002008D
:107CE8000C2A00F24881DFE812F002014601460141
:107CF8004601DB0046014601460185004601460172
:107D080046010D001A6ADFF894A122F480521A6223
:107D18001A6AD3F804C0D3F81CE022F4005242EAED
:107D280000322EF4E64E534542EA01324EF4C04E7C
:107D380000F0868051498B4200F082800021C3F810
:107D480004C0C3F81CE019641A62DA6942F40062DC
:107D5800DA615A6C79694B4DC86842F400425A643A
:107D6800036828604FF6FE7213400360F9F794FF2A
:107D78002046F9F763FF7A69D8F8003052793169FB
:107D8800A7F8441034331344BB63102280232146E0
:107D980028683A6400244FF48072FB643A4E3A65CE
:107DA8004FF40053FB65FE633C66BC647C65BC65B0
:107DB800F9F752FF7A69D8F800105279C8680C2A86
:107DC8009BBF324B03EB42022346B2F8DC302A68F1
:107DD8000343CB60136843F0020313602C4C012566
:107DE8002570FDF7B5FB2378002B3FF497AE294BA0
:107DF8001D7093E61A6ADFF8A4B022F480721A6242
:107E08001A6AD3F804A0D3F81CC022F4007242EA1C
:107E180000222CF0730C5B4542EA01224CF0600C06
:107E280013D016498B4210D00021C3F804A0C3F820
:107E38001CC0D9631A62DA6942F00802DA6188E77D
:107E48002CF4804C4CEA851C78E722F440622AF432
:107E5800405A42EA0E224AEA051AE5E76819002064
:107E680074930008CE070700EC0D002000100240B4
:107E78008510000840420F0000A24A040034014067
:107E880000100040381D00207C190020A092000836
:107E98002C1D00202D1D00203C1D0020002C014021
:107EA8001A6ADFF8F4B222F010021A621A6AD3F8DA
:107EB80004A0D3F818C022F020022CF0807C42EAFB
:107EC80000122CF4E64C5B4542EA01114CF4C04226
:107ED8003FD0A74883423CD00020C3F804A09A6151
:107EE800986319629A6942F400629A6131E71A6AE2
:107EF800DFF8A4B222F001021A621A6AD3F804A0C9
:107F0800D3F818C022F002022CF4803C02432CF073
:107F1800730C5B4542EA01024CF0600022D09449A0
:107F28008B421FD001F540618B421BD001F5806167
:107F38008B4217D001F580618B4213D00021C3F822
:107F480004A0986159631A629A6942F008029A611A
:107F5800FFE621F0C0012AF4406A41EA0E114AEA1C
:107F6800850AB9E722F00C022AF4407A4EEA0202A6
:107F780045EA0A0AE2E70C2A3FF6EBAE01A151F8FE
:107F880022F000BF517F00085B7D00085B7D000880
:107F98005B7D0008ED7E00085B7D00085B7D0008C6
:107FA8005B7D00083F7E00085B7D00085B7D000864
:107FB8005B7D0008537D000800221A867FE6198041
:107FC800DA621D857BE621F0700189B250E6694AC4
:107FD800694B122111605A685A605A685A605A6887
:107FE80042F480625A605A6822F47C125A605A68D5
:107FF80042F4E8125A601A6842F080721A601A68ED
:108008009401FCD55A685C4922F003025A605A6808
:1080180042F002025A604B6803F00C03082BFAD1B5
:10802800FFF76DB800221A6062B6544B1B6883F3E1
:108038000888534B1B689847FEE707F14003C0F1D7
:1080480004020021184401F0F8F8396C2046FEF7C4
:108058006FF87E64B8641EE50023C3EBC30305EB29
:108068008303DFF814E11969DEF8142045480A4350
:10807800CEF814204FF0000A06221A7683F819A0C9
:108088008346F9F709FE2046F9F7D8FDB8F1020F43
:1080980034BF534680233C493C4AFB64B9634FF4E0
:1080A80080734FF480615846FA633B6520224FF491
:1080B800005379652146C7F840A0C7F848A0C7F81B
:1080C80060A0BA65FB65A7F84480F9F7C5FDDBF841
:1080D80000304FF0A04A43F00103CBF80030DAF843
:1080E800083023F04053CAF80830DAF8083043F073
:1080F8008053CAF80830FCF733FFDAF8083023F069
:108108008043CAF80830DAF80830CAF80830DAF8D4
:10811800083043F00043CAF8083053469A68002AEA
:10812800FCDB9868DFF874E019491A4A20F04050DF
:108138009860986840F000509860DEF808000140A8
:1081480041F46831CEF80810D9680A4042F4005268
:10815800DA60196B08F1FF3221F00F010A431A6344
:108168004FF0A04001234FF0070B4FF01F0E1BE00C
:1081780000340140002002400010024000D8FF1FD8
:1081880004D8FF1F0800024040000050941C002043
:10819800E010FCFF07C0FFFD002C01400003005069
:1081A800584A0536B24232D0F278002AF8D003F1A4
:1081B800010C042B5FFA8CFC96F8018031795FD8AA
:1081C80003EB43035B00026B0EFA03FA22EA0A028E
:1081D80008FA03F313430363B8F1090F60D808F1F1
:1081E800FF334269426903EB43034FF0380808FA4A
:1081F80003F822EA08024261DA1C436901FA02F232
:108208001A4342613F4A0536B2426346CCD14FF029
:10821800A0421346916841F0010191601A68D207A3
:10822800FCD5DA6822F00202DA60DA6842F002026B
:10823800DA60DA6842F00102DA609A6842F0040211
:108248009A60FFF773BA304E304BC6F8E432122208
:10825800C82349F2704196E42B4E2D4BC6F8E43200
:10826800182100234AF29E327160B26006F11400B0
:108278004FF41B7219463370326100F0DEFF8BE455
:10828800092B1FD8053B03EB43035B00426B0EFA37
:1082980003FA22EA0A0208FA03F3134343639BE74B
:1082A800A8F10A028369836902EB42020BFA02F819
:1082B80023EA08038361836901FA02F21A4382619F
:1082C80063466DE70E2B0DD80A3B03EB43035B00B7
:1082D800826B0EFA03FA22EA0A0208FA03F313433E
:1082E800836379E7A3F10F0202EB42025200C36BEA
:1082F8000EFA02FA23EA0A0308FA02F21343C363E6
:108308006AE700BF941C00206819002078930008D1
:108318007093000838B5444B1A68107810F07F0045
:1083280004D1537A23F02003537238BD022878D140
:108338005388002B76D11379002B73D1537923F00E
:108348008000840004F1804101F5B8415DB20968FC
:10835800002DB4BF01F0300101F44051032860D86A
:1083680000295ED0927A002A5BD004F1804404F59B
:10837800B844002D226824DA02F03002102A4AD1CB
:1083880003F07F039A0002F1804202F5B8421368B5
:10839800590608D5136840F60F710B4043F40043A3
:1083A80043F0C0031360136823F4E04323F0400351
:1083B8009BB283F0300343F4004343F0800313601F
:1083C80029E002F44052B2F5805F24D128B9174B56
:1083D80093F82C10F9F7FEFB10E09B0003F18043A3
:1083E80003F5B8431A68520408D51A6840F60F71A5
:1083F8000A4042F4404242F080021A60236823F4A3
:10840800804323F070039BB283F4405343F400434A
:1084180043F080032360064B1B685B699847002084
:1084280038BD022038BD00BF2C18002040000020B5
:1084380050180020044B054A1B681B6A002B08BF14
:108448001346D3F8EC00704724060020B804002037
:1084580082B001B901A942B14BB113780B6012780F
:10846800101C18BF012002B070471046FBE76FF0E0
:108478000100F8E749B1FF2A85BF8A2303600A7023
:108488004FF0FF3098BF0120704708467047000042
:1084980000B510EE103A204A23F00043934283B00F
:1084A80019DDB3F1FF4F04DB30EE400A03B05DF88D
:1084B80004FB684600F07EF800F0030001281AD09B
:1084C80002280FD000B30120DDED010A9DED000A5E
:1084D80000F082FDEAE7DFED110A00F0B3F903B01E
:1084E8005DF804FBDDED010A9DED000A00F0AAF934
:1084F800B1EE400ADAE7DDED010A9DED000A00F071
:108508006BFDB1EE400AD1E7DDED010A9DED000AF1
:1085180000F098F9CAE700BFD80F493F00000000F3
:1085280000B510EE103A214A23F00043934283B07D
:108538001ADDB3F1FF4F04DB30EE400A03B05DF8FB
:1085480004FB684600F036F800F0030001281DD04F
:10855800022811D008B3DDED010A9DED000A00F0F4
:1085680071F9B1EE400AE9E70020DFED110A00F0E9
:1085780033FD03B05DF804FB0120DDED010A9DED3C
:10858800000A00F029FDB1EE400AD7E7DDED010A47
:108598009DED000A00F056F9D0E70120DDED010A53
:1085A8009DED000A00F018FDC8E700BFD80F493F4D
:1085B8000000000070B510EE103A944A23F0004411
:1085C800944286B0054668DD914A944210EE106ADE
:1085D8001ADC002BDFED8F7A8F4A24F00F0440F36A
:1085E800DD80944270EE677A66D09FED8C7A77EEE4
:1085F800C76A012077EEE67AC5ED006A77EEC77A9A
:10860800C5ED017A06B070BD854A944266DDB4F1C5
:10861800FF4F49DAE215863AA4EBC25307EE903AC7
:10862800BDEEE77ADFED7F6AB8EEC77A77EEC77AF4
:108638008DED037A67EEA67ABDEEE77AB8EEC77AD3
:1086480077EEC77A8DED047A67EEA67AF5EE407A72
:10865800F1EE10FACDED057A40F0B380B5EE407A30
:10866800F1EE10FA0CBF012302236F490191022198
:10867800009103A8294600F067F9002E12DA95ED5B
:10868800007AD5ED017AB1EE477AF1EE677A404289
:1086980085ED007AC5ED017A04E0002285ED000A37
:1086A8004260002006B070BD70EE407A0020C5ED33
:1086B800017AC5ED007AF5E7DFED5C6A9FED5C7A3B
:1086C80077EEE67A012077EEC76A77EEE67AC5EDAF
:1086D800006A77EEC77AC5ED017AE3E700F0C4FCDB
:1086E800DFED546ADFED4B5ADFED4C7AB6EE007AD7
:1086F800A0EE267ABDEEC77AF8EEC76A17EE100A22
:10870800B1EE666A1F28A6EE250A66EEA77A1DDC7A
:10871800494A411E24F0FF0352F82120934215D004
:1087280030EE677A85ED007A30EE470A002E30EE9B
:10873800670A85ED010AB5DAB1EE477AB1EE400A6B
:1087480085ED007A85ED010A4042ABE730EE677AA5
:10875800E41517EE103AC3F3C753E31A082BE1DD0B
:10876800DFED327A9FED327AF0EE405AE6EE275A84
:1087780030EE650AA6EE270AF0EE407AD6EE877A42
:1087880035EEE77A17EE103AC3F3C753E41A192CFB
:108798002CDC85ED007AB0EE650AC5E7944270EEF0
:1087A800277A10D09FED1D7A77EE876A4FF0FF3059
:1087B80077EEE67AC5ED006A77EE877AC5ED017A3D
:1087C80070E7032351E7DFED196A9FED197A77EE19
:1087D800A67A4FF0FF3077EE876A77EEE67AC5ED36
:1087E800006A77EE877AC5ED017A5BE79FED137A29
:1087F8009FED135AB0EE650AA6EE070A75EEC07A29
:10880800E6EE077AD6EE857A8AE700BFD80F493FA9
:10881800E3CB1640800FC93FD00FC93F43443537DB
:10882800800F4943000080433899000800443537D9
:1088380008A3852E84F9223FB898000800A3852E46
:1088480032318D2410EE103A23F00043B3F1485F23
:108858002CDAFDEEC07A17EE903A002B60D020EEAD
:10886800007ADFED314A9FED315ADFED315A9FED45
:10887800316ADFED317ADFED316AA7EE245AE7EE8F
:10888800055AA7EE256AE7EE067AE7EE276A66EE4E
:10889800876A60EEC00AB6EE006AE7EE260AF7EECF
:1088A800007AD7EE060A37EEE00A704720EE007A23
:1088B800DFED1D4A9FED1D5ADFED1D5A9FED1D6A24
:1088C800DFED1D7ADFED1D6A1D4AA7EE245A93429B
:1088D800E7EE055AA7EE256AE7EE067AE7EE276A7D
:1088E80066EE876AD5DD174A934214DC03F17F43AD
:1088F80007EE903AB7EE006A36EE676A60EEC00A95
:10890800F6EE005AE7EE260AD7EE257A77EEE07AF9
:1089180036EE670A7047B6EE076AF5EE027AEDE7BB
:10892800B7EE000A704700BF4ED747ADF6740F3157
:108938007CF293B4010DD037610BB6BAABAA2A3DCD
:108948009999993E0000483F2DE9F04F2DED048B91
:10895800D9B003F1FF3A0493D31E48BF131DD44C7A
:10896800669D0291DB1023EAE373194654F82560EB
:1089780006930133A2EBC3030193A1EB0A0316EBA1
:108988000A01814616D419449FEDCA7A67980131C5
:108998001CAA002BA4BF50F8234007EE904A03F10D
:1089A8000103ACBFF8EEE77AF0EE477A8B42E2ECCF
:1089B800017AEED1002EC0F20783049B44AD9C00DF
:1089C800771C1CAB05EB8707181909EB0401BAF1F2
:1089D800000FC0F27582DFEDB77A4B460246F3EC22
:1089E800016A32ED017A8B42E6EE877AF7D1E5EC3F
:1089F800017ABD4200F10400E9D106F18043013B50
:108A08009B0008AD1A1FAA18B3460396DFEDAB8A80
:108A18009FEDA98A019E07924C4405EB030844AFD9
:108A28004FEA8B0358AA1A44BBF1000F12ED140A3F
:108A380018DD07A907EB8B0260EE287AB0EE407AC2
:108A4800FDEEE77A72ED016AF8EEE77ABA42A7EE30
:108A5800C87A37EEA60ABDEEC77A17EE100A41F8B3
:108A6800040FE9D13046059300F04EFBB0EE409A72
:108A7800B4EE000A29EE000A00F0FEFAF2EE007ADF
:108A8800A0EE679A002E059BFDEEC99AF8EEE97AEA
:108A980039EE679A40F3C9800BF1FF3EC6F1080230
:108AA80055F82E1041FA02F000FA02F2891A45F838
:108AB8002E1019EE90EA8644C6F1070209EE90EAF4
:108AC8001141002951DD19EE902ABBF1000F02F186
:108AD800010209EE902A40F312822A68002A40F027
:108AE8006982BBF1010F40F32982AE4601205EF88E
:108AF800042F002A00F01E8200F1010EC2F58072D8
:108B0800F34545F8202012DD55F82E200230C2F139
:108B1800FF02834545F82E2009DD05EB8000EA18A1
:108B28000368C3F1FF0340F8043B9042F8D1002EDC
:108B38000DDD012E4FF0010240F0E7810BF1FF300F
:108B480055F8203003F07F0345F82030E7E102298B
:108B58000BD1F7EE007A37EEC99A3046B7EE000A25
:108B680000F0D2FA39EE409A0221B5EE409AF1EEC1
:108B780010FA70D1039B0BF1FF3E73450EDC0BF12D
:108B88008042013A05EB8202002052F8043942453E
:108B980040EA0300F9D1002840F09480039B013B90
:108BA80055F82330002B40F0D381079B4FF0010C80
:108BB80053F804290CF1010C002AF9D0DC440BF11C
:108BC800010EE6452FDC069A049B0EEB020103EB2F
:108BD8000B000CEB02031CAA01F1804102EB8000A0
:108BE800679A013902EB810107EB8E0E02EB830BCA
:108BF80051F8043F07EE903AF8EEE77ABAF1000F21
:108C0800E0EC017ADFED2B7A09DB4B460246F3EC08
:108C1800016A32ED017AA342E6EE877AF7D1594527
:108C2800EEEC017AE4D1E346FAE605D10BF1FF3226
:108C380055F82210091244E7F6EE007AB4EEE79AE6
:108C4800F1EE10FA80F24681B5EE409AF1EE10FA94
:108C58004FF000018ED0019C039EB0EE490A60429D
:108C6800884600F051FA9FED147AB4EEC70AF1EE87
:108C780010FAC0F28581DFED117A60EE277A23467B
:108C8800FDEEE77A0833F8EEE77A0193A7EEC70A14
:108C98000BF10103FDEEE77ABDEEC00A10EE102AD3
:108CA80045F82B2017EE902A45F823201FE000BF37
:108CB8007C9C000800000000000080430000803B0E
:108CC8000000C93F8846019955F82E20039E0839AF
:108CD800734601915AB90EF18042013A05EB8202BE
:108CE80052F80409013B08390028F9D0019101988C
:108CF8000393B7EE000A00F007FA039B002BC0F2BB
:108D08004A819F0044AAD01907F1040E1FED157A75
:108D180005EB0E02011D72ED017AF8EEE77AAA4220
:108D280067EE807A20EE070A61ED017AF3D11FED34
:108D38001C6A05460DF5867C0024002EC0F2DC80F6
:108D4800A348DFEDA47A2946B0EE467A002203E074
:108D5800A24208DCB0EC017AF1EC016A01329642D9
:108D6800E7EE267AF4DA043D58AA02EB8402654558
:108D780042ED287A04F10104DFD1669A032A5AD811
:108D8800DFE802F08C626202002B40F3018158AAEE
:108D98003A4430A912ED287A3A1D0A4431A83944D8
:108DA80051ED017A77EE876A77EEE67A77EE877A81
:108DB800B0EE667A62ED017A824261ED016AEFD126
:108DC800012B40F3E58058AB3B4430AA13ED287AD9
:108DD8003B1D32A917441A4457ED017A77EE876A8A
:108DE80077EEE67A77EE877AB0EE667A62ED017A08
:108DF800914267ED016AEFD130A9DFED767A0B4435
:108E080033ED017A9A4277EE877AF9D14346002BFF
:108E180000F0AE80DDED306A9DED317A029AF1EE18
:108E2800677AF1EE666AB1EE477AC2ED027AC2ED70
:108E3800006A82ED017A19EE903A03F0070059B002
:108E4800BDEC048BBDE8F08F3A1D30A9DFED617AE7
:108E58000A4432ED017A8A4277EE877AF9D142469E
:108E6800002A78D0DDED306A029AB1EE677A002BDD
:108E780076EEE77A82ED007A0ADD31A90122B1ECBB
:108E8800017A0132934277EE877AF8DA43460BB1DA
:108E9800F1EE677A029BC3ED017ACCE730ABDFEDE8
:108EA8004D7A9E443EED017A734577EE877AF9D183
:108EB80043460BB1F1EE677A029BC3ED007ABAE73D
:108EC800DFED447AE5EC017ABD4200F104007FF45D
:108ED8007EAD92E519EE902ABBF1000F02F1010276
:108EE80009EE902AC8BF02213FF7F7ADF7EE007AE6
:108EF80037EEC99A022138E6DFED367A33E7002EDD
:108F08001EDD0022012E3FF419AE022E07D10BF10F
:108F1800FF3055F8203003F03F0345F82030022990
:108F28007FF423AEF7EE007A37EEC99A002A3FF4B1
:108F38001CAE12E6013083457FF4D9AD002EE1DC8A
:108F480002297FF412AEF7EE007A37EEC99A0CE6E2
:108F58004FF0010C32E69DED307A029A002BC2EDFB
:108F6800007A77EE677A88DC029BC3ED017A62E7C4
:108F78000298309A319BC0ED027A026043605AE74A
:108F8800BDEEC00A5B4610EE102A45F82B20AEE66F
:108F9800DFED107A3AE7669A032A3FF64CAF01A153
:108FA80051F822F0CB8F0008C58F0008C58F000844
:108FB800998F00084FF0010E00209FE5DFED057A3C
:108FC8004DE7DFED047A73E7049B9C0015E500BFCD
:108FD800549C00080000000010EE103A23F00043F3
:108FE800B3F1485F04DAFDEEC07A17EE903A23B386
:108FF80060EE007A9FED155ADFED155A9FED156A60
:10900800DFED156A9FED157AE7EE855A20EE275AAF
:10901800A7EEA56AE7EE866AA7EEA67A70B127EEF4
:10902800457AF6EE006AA0EEA67ADFED0D6AD7EE75
:10903800870AE5EE260A30EE600A7047DFED096A16
:10904800E7EE876AA5EE260A704700BFD3C92E2F20
:10905800342FD7B21BEF3836010D50B98988083C38
:10906800ABAA2A3EABAA2ABE10EE103A23F0004360
:1090780000EE103A704700BF10EE102A22F00041AF
:10908800CB0D7F3B162B17DC002B10EE100A19DBDB
:109098001A4919410A4222D0DFED197A70EE277A6F
:1090A800F5EEC07AF1EE10FA19DD002A18DB20EA95
:1090B800010300EE103A7047B1F1FF4F0FD330EEC5
:1090C800000A7047DFED0E7A70EE277AF5EEC07A67
:1090D800F1EE10FA03DD002A08DB9FED0A0A70475B
:1090E8004FF4000242FA03F31844E0E70029FFEEC8
:1090F800007A18BFB0EE670A704700BFFFFF7F0015
:10910800CAF249710000000008B510EE103A33F0B9
:1091180000422DED028B11D0B2F1FF4F11D2B2F502
:10912800000F13D3D20D0244FE2A2EDC002A1ADDCA
:1091380023F0FF4343EAC25300EE103ABDEC028B22
:1091480008BDBDEC028B30EE000A08BD1D4BDFEDFB
:109158001E7A984220EE270A22DB10EE103AC3F35B
:10916800C752193ADFE712F1160F1EDA4CF25033E4
:1091780098420ADC9FED158AF0EE400AB0EE480AE4
:1091880000F02AF820EE080AD8E79FED118AF0EEE1
:10919800400AB0EE480A00F01FF820EE080ACDE7B2
:1091A800DFED0A0A20EE200AC8E7193223F0FF4350
:1091B80043EAC253DFED077A00EE103A20EE270AA1
:1091C800BCE700BFB03CFFFF0000004C6042A20DAE
:1091D800CAF249710000003310EE103A10EE902ADE
:1091E80023F0004302F00042134300EE103A7047A8
:1091F80010B5431E0A44914200D110BD11F8014B2D
:1092080003F8014FF7E7884210B501EB020303D8D2
:10921800421E99420CD110BD9842F9D28118D21A37
:10922800D34200D110BD13F8014D01F8014DF7E705
:1092380011F8014B02F8014FEBE702440346934251
:1092480000D1704703F8011BF9E72DE9F041064604
:109258000F4600EB0208464519D016F8014BFFF7F8
:10926800E9F8204417F8015B437803F00303012B66
:1092780008BF2034FFF7DEF82844437803F00303DF
:10928800012B08BF2035601B04D1002DE3D100203D
:10929800BDE8F081BDE8F081000000000038014021
:1092A80000000000000000001A27350019263400CD
:1092B8004E07255050000000020000000048004002
:1092C80000000000000000002B3B00002A3A0000CC
:1092D80072072740500000000000000000300140E5
:1092E800152316241725054C0100000000380040FE
:1092F8002D232E242F25056E02000000003C00407F
:10930800233A243B253C066F00000000005400402F
:109318001F26281E272975000000000000000000F5
:109328000000000000000000000000008025000090
:10933800004B00000096000000E1000000C20100A0
:109348000084030090D00300801A0600000807007C
:1093580020A1070000100E0040420F0060E3160035
:1093680080841E0070B025001D100008810F0008C1
:10937800CD0E0008000200000000000000040000FC
:1093880000000000000800000000000000100000BD
:10939800181E0020181F0020FFFF0000000000001A
:1093A800002C01404B1B000000000040601C000026
:1093B80000040040611D000000080040621E00001B
:1093C8000010004064000000001400406500000028
:1093D800003401404D2E00000040014050180000AC
:1093E800004401405119000000480140521A000091
:1093F8003132333435360000F1250008F1250008F4
:109408000D660008F1250008F1250008F12500087F
:10941800F125000859660008F1250008F125000823
:10942800F1250008F1250008F1250008F1250008BC
:10943800591A0008CD1A0008511B0008C91D000858
:10944800C11A0008891A00086D1A0008611A000874
:109458005D1A0008191B0008511A00082931000874
:109468007130000865300008A13100088530000817
:109478007D30000881300008493100086930000853
:1094880021310008140002000010203031310000A2
:10949800FFFFFFFFFFFF040000001300B5100008E6
:1094A80035420008691100081511000845430008F5
:1094B800511100088542000800000000000000006B
:1094C8000000000000040040200804010200000021
:1094D8001C0002400100000000040040210C0401AF
:1094E8000200000030000240020000000044014079
:1094F80024000401010000006C0002400500000087
:1095080000480140250004010A00000080000240D4
:1095180006000000002C0140180020000600000092
:109528001C000240010000000000000000000000D4
:109538000000000000000000000000000000000023
:109548000000000000000000000000000000000013
:109558000000000000000000000000000000000003
:1095680000000000000000000000000000000000F3
:1095780000000000000000000000000000000000E3
:1095880000000000000000000000000000000000D3
:1095980000000000000000000000000000000000C3
:1095A80000000000000000000000000000000000B3
:1095B800000000006E0A010001069411102702093C
:1095C800941110270301E4578813000000090408C8
:1095D80003090607010609070802060001001234FC
:1095E80056789ABC000000001001110212031304FF
:1095F8001401150216031704200C2101220C2C0358
:109608002D052E042F05300631073208330934059D
:10961800350B000C000D000700080009000A000BBC
:10962800000D00060002000E000F001000030001EC
:109638000002000A64050000120100020200004056
:109648008304405700020102030100003203530063
:1096580054004D00330032002000560069007200AB
:109668007400750061006C00200043004F004D003D
:10967800200050006F0072007400200020000000DD
:109688002603530054004D006900630072006F0008
:1096980065006C0065006300740072006F006E0066
:1096A800690063007300000004030904040100005A
:1096B80009024300020100C032090400000102024D
:1096C8000100052400100105240100010424020200
:1096D8000524060001070582030800FF09040100AC
:1096E800020A000000070503024000000705810286
:1096F80040000000434C464C00000000534F4633E6
:10970800000000004F6374203130203230313700C0
:1097180030373A32323A31350000000036303538C9
:10972800386533613700000057414954494E472096
:10973800464F522046430000322E312E30000000A2
:10974800562573004F53440053595354454D000058
:1097580053455249414C0000424154544552595FC7
:10976800564F4C5441474500424154544552595F65
:1097780043555252454E5400424154544552595F44
:10978800414C4552545300005452414E53504F4E91
:10979800444552004F53445F534C41564500000026
:1097A800534F4633004300504F534958002E000092
:1097B8002020202020202020202828282828202079
:1097C8002020202020202020202020202020202091
:1097D8008810101010101010101010101010101009
:1097E80004040404040404040404101010101010E9
:1097F80010414141414141010101010101010101C2
:1098080001010101010101010101011010101010F5
:109818001042424242424202020202020202020292
:1098280002020202020202020202021010101020BA
:109838000000000000000000000000000000000020
:109848000000000000000000000000000000000010
:109858000000000000000000000000000000000000
:1098680000000000000000000000000000000000F0
:1098780000000000000000000000000000000000E0
:1098880000000000000000000000000000000000D0
:1098980000000000000000000000000000000000C0
:1098A80000000000000000000000000000000000B0
:1098B800000FC93F000F494000CB9640000FC94038
:1098C8000053FB4000CB164100ED2F41000F4941EA
:1098D8000031624100537B41003A8A4100CB9641F6
:1098E800005CA34100EDAF41007EBC41000FC941BF
:1098F80000A0D5410031E24100C2EE410053FB41D6
:1099080000F20342003A0A420083104200CB16429A
:1099180000141D42005C234200A5294200ED2F429D
:1099280000363642007E3C4200C74242000F4942A0
:10993800A2000000F9000000830000006E00000093
:109948004E0000004400000015000000290000003F
:10995800FC0000002700000057000000D1000000B4
:10996800F500000034000000DD000000C000000029
:10997800DB00000062000000950000009900000074
:109988003C0000004300000090000000410000007F
:10999800FE0000005100000063000000AB00000062
:1099A800DE000000BB000000C500000061000000F0
:1099B800B7000000240000006E0000003A0000001C
:1099C800420000004D000000D2000000E00000004E
:1099D80006000000490000002E000000EA00000018
:1099E80009000000D1000000920000001C000000E7
:1099F800FE0000001D000000EB0000001C0000003D
:109A0800B100000029000000A70000003E0000008F
:109A1800E80000008200000035000000F5000000AA
:109A28002E000000BB00000044000000840000007D
:109A3800E90000009C000000700000002600000003
:109A4800B40000005F0000007E000000410000003C
:109A58003900000091000000D60000003900000025
:109A6800830000005300000039000000F4000000EB
:109A78009C000000840000005F0000008B000000D4
:109A8800BD000000F9000000280000003B000000B5
:109A98001F000000F800000097000000FF00000011
:109AA800DE00000005000000980000000F00000024
:109AB800EF0000002F000000110000008B000000E4
:109AC8005A0000000A0000006D0000001F0000009E
:109AD8006D000000360000007E000000CF0000008E
:109AE80027000000CB00000009000000B7000000BC
:109AF8004F000000460000003F0000006600000024
:109B08009E0000005F000000EA0000002D00000039
:109B18007500000027000000BA000000C700000020
:109B2800EB000000E5000000F10000007B000000F1
:109B38003D0000000700000039000000F7000000A9
:109B48008A0000005200000092000000EA000000B5
:109B58006B000000FB0000005F000000B100000087
:109B68001F0000008D0000005D00000008000000DC
:109B7800560000000300000030000000460000000E
:109B8800FC0000007B0000006B000000AB00000040
:109B9800F0000000CF000000BC0000002000000022
:109BA8009A000000F4000000360000001D000000CC
:109BB800A9000000E300000091000000610000001F
:109BC8005E000000E60000001B0000000800000026
:109BD8006500000099000000850000005F0000009B
:109BE80014000000A0000000680000004000000011
:109BF8008D000000FF000000D80000008000000079
:109C08004D00000073000000270000003100000034
:109C180006000000060000001500000056000000C5
:109C2800CA00000073000000A8000000C90000007E
:109C380060000000E20000007B000000C00000009F
:109C48008C0000006B0000000000C93F0000F039E4
:109C58000000DA370000A2330000842E0000502BE9
:109C68000000C2270000D0220000C41F0000C61B4D
:109C7800000044170400000007000000090000006D
:109C880012000200400B0020700B002000000000B2
:109C9800B49D000813000400D80D0020E00D00203A
:109CA80000000000B89D0008FE010800E80E002032
:109CB800E00E002000000000BD0E000801020500B3
:109CC8000C11002058150020000000008D560008D7
:109CD8000D001C00FC150020581800200000000092
:109CE800C559000802020300F0150020741800206E
:109CF8000000000000000000F9010400C418002062
:109D0800C01800200000000075420008FD011E0078
:109D1800E8180020C8180020000000005D42000874
:109D280011000C005C190020541C002000000000E9
:109D38007D590008000104009C1C0020901D002093
:109D480000000000BC9D00080B100C00741C0020D3
:109D5800941D002000000000C09D000802010300BF
:109D68001C1D0020A01D0020000000009D560008BA
:109D780006020800AC1D0020A41D00200000000001
:109D88007B5F000808020900C01D0020B41D0020E8
:109D980000000000515F0008F7010600D81D0020F0
:0C9DA800D01D002000000000CC9D000831
:109DB4000001000000212000900100002B21231E3F
:0E9DC4000101000001000A0100000100000082
:109DD200E0010800FFFF0000000000000102030490
:109DE200010203040607080901000200040006003C
:109DF20008000A000C001000200040008000000152
:109E0200000000000000000000C201000000080085
:109E12005568000865660008D5650008D165000828
:109E2200716500084D650008BD64000829650008D9
:109E320005650008CD640008000000004000000035
:109E4200F1250008F5650008F1250008F125000854
:109E5200F1250008F1250008F1250008F125000888
:109E6200E96500080000024008000240000000000E
:109E7200000B0000010000000000000000000000D4
:109E8200000002401C00024000000000040C000020
:109E9200010000000000000000000000000002407D
:109EA2003000024000000000080D00000100000028
:109EB20000000000000000000000024044000240D8
:109EC200000000000C0E0000010000000000000075
:109ED20000000000000002405800024000000000A4
:109EE200100F000001000000000000000000000050
:109EF200000002406C00024000000000141000004C
:109F0200010000000000000000000000000002400C
:109F12008000024000000000181100000100000053
:109F2200000000000000000000040240080402409B
:109F320000000000003800000200000000000000E5
:109F420000000000000402401C0402400000000067
:109F520004390000020000000000000000000000C0
:109F6200000402403004024000000000083A0000F1
:109F72000200000000000000000000000004024097
:109F820044040240000000000C3B000002000000FC
:109F920000000000000000000004024058040240DB
:109FA20000000000103C0000020000000000000061
:109FB20000000000509700080000000000000000B0
:109FC20079580008A086010004000000000000008B
:109FD200000000000000000000000000000000007F
:109FE200000000000000000000000000000000006F
:109FF200000000000000000000000000000000005F
:10A00200000000000000000000000000000000004E
:10A01200000000000000000000000000000000003E
:10A02200000000000000000000000000000000002E
:10A03200000000000000000000000000000000001E
:10A04200000000000000000000000000000000000E
:10A0520000000000000000000000000000000000FE
:10A0620000000000000000000000000000000000EE
:10A0720000000000000000000000000000000000DE
:10A0820000000000000000000000000000000000CE
:10A0920000000000000000000000000000000000BE
:10A0A20000000000000000000000000000000000AE
:10A0B20000000000000000005897000800000000A7
:10A0C200850E000889010008102700000600000024
:10A0D200000000000000000000000000000000007E
:10A0E200000000000000000000000000000000006E
:10A0F200000000000000000000000000000000005E
:10A10200000000000000000000000000000000004D
:10A11200000000000000000000000000000000003D
:10A12200609700080000000000000000A15700082E
:10A13200204E0000030000000000000000000000AC
:10A14200000000000000000000000000000000000D
:10A1520000000000709700080000000000000000EE
:10A16200AD560008204E0000030000000000000071
:10A1720000000000000000000000000000000000DD
:10A1820000000000000000008097000800000000AE
:10A1920000000000DD6D0008400D03000300000018
:10A1A20000000000000000000000000000000000AD
:10A1B200000000000000000000000000909700086E
:10A1C2000000000000000000A9580008A00F0000D5
:10A1D200010000000000000000000000000000007C
:10A1E200000000000000000000000000000000006D
:10A1F2009C97000800000000D11A0008251A0008E8
:10A202001A410000050000000000000000000000EC
:10A21200000000000000000000000000000000003C
:10A2220000000000B09600080400000088960008B4
:10A23200260000005496000832000000840400202A
:10A242001A000000B896000843000000409600087B
:10A25200120000001A03530054004D003300320074
:10A2620000000000000000000000000000000000EC
:10A2720001000000000000000000000001020304D1
:10A28200060708090100000043000000000000006A
:10A2920000000000000000000000000000000000BC
:10A2A2000000000000000000430000000000000069
:10A2B200000000000000000000000000000000009C
:10A2C2000000000000000000430000000000000049
:10A2D200000000000000000000000000000000007C
:10A2E2000000000000000000430000000000000029
:10A2F200000000000000000000000000000000005C
:10A302000000000000000000430000000000000008
:10A31200000000000000000000000000000000003B
:10A3220000000000000000004300000000000000E8
:10A33200000000000000000000000000000000001B
:10A3420000000000000000004300000000000000C8
:10A3520000000000000000000000000000000000FB
:10A3620000000000000000007D84000859840008FD
:10A3720000000000B7970008B5970008B6970008DC
:10A38200B6970008B6970008B6970008B697000877
:10A39200B6970008B6970008B6970008B697000867
:10A3A200FFFFFFFFFFFFFFFFFFFFFFFFFFFF0000B9
:10A3B2000100415343494900000000000000000031
:10A3C200000000000000000000000000000000008B
:10A3D2000000415343494900000000000000000012
:10A3E200000000000000000000000000000000006B
:10A3F200000000002806002000000000000000000D
:10A40200000000000000000000000000000000004A
:10A41200000000000000000000000000000000003A
:10A42200000000000000000000000000000000002A
:10A43200000000000000000000000000000000001A
:10A44200000000000000000000000000000000000A
:08A45200000000000000000002
:0400000508000000EF
:00000001FF
